:100000005062040000000000FFFFFF00FFFFFF0040
:10001000FFFFFF00FFFFFF00FFFFFF00FFFFFF00EC
:10002000FFFFFF00FFFFFF00FFFFFF00FC020000DB
:10003000FFFFFF00FFFFFF00BC020000FFFFFF000B
:10004000FFFFFF00FFFFFF00FFFFFF00B001000008
:10005000FFFFFF004A030000FFFFFF00FFFFFF005C
:10006000FFFFFF00FFFFFF00FFFFFF006E02000029
:1000700020020000FFFFFF00FFFFFF00FFFFFF0067
:10008000FFFFFF00FFFFFF0000010000FFFFFF0078
:10009000FFFFFF00FFFFFF00FFFFFF00FFFFFF006C
:1000A000FFFFFF00FFFFFF00FFFFFF00FFFFFF005C
:1000B000FFFFFF00FFFFFF00FFFFFF00FFFFFF004C
:1000C000FFFFFF00FFFFFF00FFFFFF00FFFFFF003C
:1000D000FFFFFF00FFFFFF00FFFFFF00FFFFFF002C
:1000E000FFFFFF00FFFFFF00FFFFFF00FFFFFF001C
:1000F000FFFFFF00FFFFFF00FFFFFF00FFFFFF000C
:10010000FFFFFF00FFFFFF00FFFFFF00FFFFFF00FB
:10011000FFFFFF00FFFFFF00FFFFFF00FFFFFF00EB
:10012000FFFFFF00FFFFFF00FFFFFF00FFFFFF00DB
:10013000FFFFFF00FFFFFF00FFFFFF00FFFFFF00CB
:10014000FFFFFF00FFFFFF00FFFFFF00FFFFFF00BB
:10015000FFFFFF00FFFFFF00FFFFFF00FFFFFF00AB
:10016000FFFFFF00FFFFFF00FFFFFF00FFFFFF009B
:10017000FFFFFF00FFFFFF00FFFFFF00FFFFFF008B
:10018000FFFFFF00FFFFFF00FFFFFF00FFFFFF007B
:10019000FFFFFF00FFFFFF00FFFFFF00FFFFFF006B
:1001A000FFFFFF00FFFFFF00FFFFFF00FFFFFF005B
:1001B000FFFFFF00FFFFFF00FFFFFF00FFFFFF004B
:1001C000FFFFFF00FFFFFF00FFFFFF00FFFFFF003B
:1001D000FFFFFF00FFFFFF00FFFFFF00FFFFFF002B
:1001E000FFFFFF00FFFFFF00FFFFFF00FFFFFF001B
:1001F000FFFFFF00FFFFFF00FFFFFF00FFFFFF000B
:100200000200FA003600F800801F7800200020006D
:100210000C000900B01F7800C01080006200600070
:100220004101DE006000510040003A00C010800033
:10023000610160003B003200E0108000000F780098
:10024000020F200060004700100261000209200038
:10025000020052001A003600E00247001500780044
:100260004500DE00650050004101DD0040F920003E
:1002700002024000C4628800050078001000780087
:100280006F016000400620000010B800000A7800EE
:100290000500780010007800700160000400320052
:1002A000F0FF2F00D06288005C0104000000000015
:1002B00010002000D06288008E01040000000000C1
:1002C00060024700140078004400DE006F01600007
:1002D000A00020000011B800040078001000780091
:1002E0006F00600000014100C06280001008410002
:1002F000C062800010017800A0C520001091B900F4
:10030000C062800002087800A27C8000C0C5200086
:1003100060081100B07C8000F062880016010400C3
:10032000000000009C01040000000000D2FF2F002C
:100330008021200010086100F2EF2F0060082000EB
:1003400010086100A00120000C0009004F10780087
:100350004F0078003600F9000080FA0000400600E7
:100360003600F800801F7800200020000C000900F3
:10037000B01F78007010800062006000C102DE00D3
:100380006080520022003A0070108000E10260009C
:100390001D00320005C6200000D0200090824200DF
:1003A00090108000804A780000688000E1024000E0
:1003B00005688800020A2000110009008282D80026
:1003C0000100780000688800E1024000020A200075
:1003D000110009008282D8000100780026D0200098
:1003E0009602500006003A001000200020688800A5
:1003F00000002000106888000000200000688800CD
:10040000C4010400000000000E020400000000000F
:10041000D5FF2F00E020200010886200F5DF2F00BC
:100420004008200010886200A00120000C00090094
:100430004F1078004F0078003600F90000400600A9
:100440003600F800801F7800200020000C00090012
:10045000B01F78005E61AE003802040000000000AA
:10046000E00A8000010020002A02040000000000D1
:1004700061E72000C8A2AE004802040000000000AE
:1004800080087800910098006002040000000000DD
:100490000001780011005100306888008000EB00F6
:1004A00041688800516880000100E00004003A00C3
:1004B000616880000100E00001003200C00E880089
:1004C0008640A900A00120000C0009004F10780010
:1004D0004F0078003600F900004006003600F800B2
:1004E000801F7800200020000C000900B01F780059
:1004F0005A61AE008602040000000000C00A8000BD
:1005000001002000780204000000000021E7200024
:10051000C882AE0096020400000000008008780047
:1005200091009800AE020400000000000001780075
:1005300011005100706888008000EB00816888001D
:10054000516880000100E00004003A00616880000A
:100550000100E00001003200B00E88008620A900F2
:10056000A00120000C0009004F1078004F00780017
:100570003600F900004006003600F800801F7800C1
:10058000200020000C000900B01F78004661AE007A
:10059000D402040000000000200A800001002000B6
:1005A000C602040000000000A1E72000D422AE0033
:1005B000E402040000000000800878009100980028
:1005C000EE0204000000000000017800110051005C
:1005D000906888000000EB00A06888008480A90073
:1005E000A00120000C0009004F1078004F00780097
:1005F0003600F900004006003600F800801F780041
:10060000200020000C000900B01F78004261AE00FD
:100610001403040000000000000A80000100200014
:100620000603040000000000E1E72000D402AE0051
:100630002403040000000000800878009100980066
:100640003C0304000000000000017800110051008C
:10065000B06888008000EB00C168880051688000A5
:100660000100E00004003A00616880000100E00041
:1006700001003200D00E88008420A900A0012000D3
:100680000C0009004F1078004F0078003600F90088
:10069000004006000200FA003600F800801F7800D3
:1006A000200020000C000900B01F7800001480001A
:1006B000D068880010148000E06888002014800052
:1006C000F06888003014800000698800F2688000BB
:1006D000CF91DE0020D22000101841001090490078
:1006E00002698000CF91DE0060D220001018410026
:1006F00010904900506980006102400054698800F0
:10070000823E20000200520028003500526980001D
:10071000CF91DE0010698000216980000002EB00AB
:10072000361E070044C42000140150000207980040
:100730006269880052698000CF91DE0030698000D4
:10074000416980000002EB002C1E070070698800E0
:1007500000002000CF80DE003069880041698800F9
:100760000000200001002000106988002169880035
:1007700000002000506988000E01900060005100C8
:1007800002003D000000200060698800626980006E
:10079000CF91DE0000D320001018410010904900D6
:1007A0001200200040D3200010484100F27F2F00AB
:1007B0004008200010086100A00120000C00090082
:1007C0004F1078004F0078003600F9000080FA00E2
:1007D0000040060001002800C020200010887000A2
:1007E00001402000E020200010887000000006007A
:1007F0000000FA00711080000010200000806000EE
:10080000C800DE000100E00002003A00FA03040024
:100810000000000068005700104078000080FB00D6
:10082000801088000080FA00000006000000000030
:100830000000000090108000000006007010800092
:1008400061006000000006007110800000102000B0
:1008500000806000C800DE000100E00003003A00F4
:100860000000000024040400000000000000060056
:100870000C00FA00803F2000B06988006041200031
:10088000C0698800E0412000D06988004042200013
:10089000E0698800A03E2000F0698800C055200073
:1008A000006A880000002000601088000000280016
:1008B0007010880048000700000F780011079800AA
:1008C000823E2000CF91DE00EC2E0700200798002A
:1008D00031079800000F780011079800660020008B
:1008E000CFB3DE006A02570034017800A40178001B
:1008F0000603E900030035000201D0008381D20025
:10090000FBFF370042079800530798000002EB00F6
:100910008E1D07002E029000BE0290004E01900036
:10092000DE0190002007980031079800040078004D
:10093000850078000002EB00B01D0700000F780072
:100940001107980012002000CF91DE004E009000A9
:10095000DE00900000027800810278000201E900C8
:10096000030035008502D1000482D300FBFF37006D
:100970002E019000BE019000040051000580590036
:100980000500360012002000CF91DE006000470015
:1009900010184100109049006001470032007800B3
:1009A000A200780061005000E0805800000F78003D
:1009B00011079800A0108800D2FF2F00E02020002F
:1009C0001008610083FF07000D0007000C000700FE
:1009D0000080FA00000006000088230011002000BB
:1009E000000006000100280060212000108870002F
:1009F00001402000802120001088700000000600C7
:100A0000E0462000801F7800A0072000801F7800AB
:100A10000C2C07004F00B100000006000000FA0097
:100A2000C11080000010200000806000C800DE00BF
:100A30000100E00002003A00100504000000000080
:100A400068005700104078000080FB00D01088003C
:100A50000080FA0000000600000000000000000016
:100A6000E010800000000600C010800061006000FF
:100A700000000600C110800000102000008060000F
:100A8000C800DE000100E00003003A0000000000A2
:100A90003A0504000000000000000600F1FF2700F6
:100AA0006021200010886000F1BF2F00802120000D
:100AB0001088600000000600F1FF2700C020200021
:100AC00010886000F1BF2F00E02020001088600037
:100AD000000006000C00FA00E0502000B069880019
:100AE000C0522000C069880040532000D0698800AF
:100AF000A0532000E0698800204F2000F0698800A2
:100B0000E0542000006A880000002000B010880037
:100B100000002800C0108800AFFF0700000F780019
:100B200011079800823E2000CF91DE00532E07006F
:100B30002007980031079800000F780011079800EF
:100B400066002000CFB3DE006A025700340178004F
:100B5000A40178000603E900030035000201D0007B
:100B60008381D200FBFF37004207980053079800AB
:100B70000002EB00F51C07002E029000BE02900060
:100B80004E019000DE019000200798003107980088
:100B900004007800850078000002EB00171D0700B4
:100BA000000F78001107980012002000CF91DE009E
:100BB0004E009000DE009000000278008102780074
:100BC0000201E900030035008502D1000482D30050
:100BD000FBFF37002E019000BE0190000400510081
:100BE000058059000500360012002000CF91DE007C
:100BF0006000470010184100109049006001470054
:100C000032007800A200780061005000E0805800B7
:100C1000000F780011079800F0108800D2FF2F0015
:100C200080212000100861006EFF070074FF07009C
:100C300073FF07000080FA00000006004003200058
:100C40004015880040042000001588004041200025
:100C500010158800301020002015880000002000AA
:100C600030158800B01C200050158800B0FF2F0000
:100C70003016880000002000A0168800F0FF2F002A
:100C80009016880000002000C01688000000200098
:100C9000F016880000000600F1F32F00E02020008D
:100CA0001088600001022000800920009080680008
:100CB0000007200080806000800920001088680004
:100CC000F1DF2F0040082000108860000120200084
:100CD000C008200010887000F1F32F008021200050
:100CE0001088600011002000000A200010806800B9
:100CF000E7006000000A2000108868000110200052
:100D0000E0082000108870000000200030088800F3
:100D10000001280080088800E00420007008880096
:100D2000000020005008880000012800900888007A
:100D300001002800002A200010887000F17F2F0099
:100D4000400820001088600001802000C0082000BA
:100D50001088700001082000A01520001088700085
:100D600011002000A015200010806800E70060003E
:100D7000A01520001088680001022000C009200092
:100D8000908068000007200080806000C00920007B
:100D900010886800D1FF2F006008200010886000D4
:100DA00021002000E00820001088700001082000C9
:100DB000E01520001088700011002000E0152000D0
:100DC00010806800E7006000E015200010886800CF
:100DD00001202000C00920009080680000702000E1
:100DE00080806000C009200010886800B1FF2F00DB
:100DF000600820001088600041002000E00820000A
:100E00001088700001082000201420001088700055
:100E1000110020002014200010806800E70060000E
:100E200020142000108868000102200040092000E2
:100E3000908068000007200080806000400920004A
:100E400010886800D1FF2F00400820001088600043
:100E500021002000C0082000108870000108200038
:100E60006014200010887000110020006014200021
:100E700010806800E700600060142000108868009F
:100E8000210020006009200010806800E700600059
:100E90006009200010886800F1FE2F004008200043
:100EA0001088600001012000C00820001088700038
:100EB000000006000000FA00F1FB2F0000222000D5
:100EC000108860000011800062006000C100DE0038
:100ED0000100E00002003200620704000000000090
:100EE0006800570010007800201188000011800071
:100EF000E100600002003A007607040000000000F4
:100F0000201180000080FA00000006000000FA00B6
:100F10000100280000222000108870000080FA00E4
:100F2000000006000000FA00F1FF27000022200068
:100F3000108860000080FA00000006000000FA003F
:100F4000A0752000106A880060782000206A880060
:100F500020792000306A88006800570090007800EF
:100F60006A005700908070006C00570090807000FD
:100F70006E005700908070007000570090807000E5
:100F8000720057009080700074005700108170004C
:100F9000F60057002022200011087100F1FB2F00FD
:100FA000002220001088600001002800002220009C
:100FB000108870000080FA00000006000A00FA00A5
:100FC00060004700A1D82E000900090031587800C0
:100FD000E0222000801F7800D0032000801F7800CE
:100FE000982A07004F00B10060004700801F78007A
:100FF0009C1A07002F00B100E0462000801F7800F7
:10100000A0072000801F78008E2A07004F00B10043
:101010006800570010007800A01088000080FA00D7
:10102000000006000200FA00F0FF2F00000F780019
:101030000468800023D02000130052000E0032000C
:1010400003C6200020D0200090814100134078008A
:101050000080FB00000F780010688000E101400074
:1010600013688800020A2000110009008281D8005C
:1010700001007800106888001E0078000080FA00E7
:10108000000006000168800020D020001080500081
:1010900002003A000000200001003700100020008C
:1010A000000006000000FA006C0157009240780032
:1010B00010002000124910000104E0001D00320061
:1010C0004EB897009040780060C050000700320092
:1010D0003EB997004EB897009040780012C050007B
:1010E00002003A008A08040000000000CEB8970011
:1010F0003EB89700104178000100780090407800D9
:101100008180FB000281FB0002007800008050001B
:1011100009003700110020006800570010884000C7
:10112000110020006A005700108840005408040095
:1011300000000000000020000080FA00000006000F
:101140000400FA00680057001000780010079800AB
:1011500000002000000F7800620047009000780037
:10116000608050001100360011002000620047002E
:10117000108810001E017800110020006000470058
:10118000108840006A0057001000410010417800AC
:10119000C10220000140510002003200BA080400E0
:1011A00000000000AC080400000000001E007800F1
:1011B0000080FA00000006002A00FA0070004700D4
:1011C00041D92E001300090031587800000020009A
:1011D0003007980000002000010020004007980020
:1011E00051079800D0CC2C00C1DC23006007980088
:1011F00071079800000020002017980000002000D0
:10120000000F780060004700100178007300510063
:101210001C003D0068005700100178006000470086
:101220001000410010427800D2022000024052001B
:101230001400390068005700100178006000470072
:10124000100041001042780092032000024052003A
:101250000C003E0070004700E0024700150240000D
:101260006800570010017800050078001000410068
:10127000104A780010002000950A4000020904007E
:1012800000000000F00247006002470014814200A5
:101290000000200000497800040078001000780069
:1012A00010079800040078001000780020079800CC
:1012B0000500780010427800D2022000024052005F
:1012C00002003A0010002000300798006600470036
:1012D00010007800000F78006000470010027800CE
:1012E000620147001200520018003D0070014700E3
:1012F000600047001000410010427800E202200028
:10130000024052000C003A006001470012007800D1
:10131000200798000200780010027800660147005C
:101320001200520002003A00F0FF2F002007980040
:10133000A609040000000000120020006000470021
:10134000100841006C09040000000000F4FF2F00A9
:1013500064014700120012002A00320064004700B6
:1013600010017800600047006108510060004700EC
:10137000100278006601470012005200210035007B
:101380006E009000FE009000020020000312240076
:10139000142A07003017980041179800600798003A
:1013A000710798007001470060004700100041007D
:1013B000104178000281FB00000320000000510072
:1013C000CF80DE000081EB00AB2907003E119000CA
:1013D000CE119000032A070068024700340178000C
:1013E000A4017800D42A070040079800510798000C
:1013F000120020006000470010081100B609040028
:10140000000000000000200001F8230060079800A1
:1014100071079800620047001000780061025000D8
:1014200064014700120012003D003200F4FF2F005B
:10143000640147001200120003003A0066004700F2
:101440001000780020079800000020002017980066
:1014500066004700100178006000510002003A0069
:101460001000200020179800640047001001780049
:1014700066004700100241004202200002014700BE
:101480006000470012084200600047001002780028
:10149000620147001200520021003D0002002000BE
:1014A000031224006E009000FE009000582B0700ED
:1014B000301798004117980060079800710798004E
:1014C00070014700600047001000410010417800A3
:1014D0000281FB000003200000005100CF80DE00ED
:1014E0000081EB00642907003E119000CE119000AE
:1014F000BC2907006802470034017800A401780085
:101500008D2A07004007980051079800120020001C
:101510006000470010084100440A04000000000079
:1015200066004700100178006100510007003A0092
:101530004E009000DE0090000200200003F82B0017
:10154000A829070040079800510798004E00900016
:10155000DE0090000080FA00000006000600FA009D
:10156000CEB89700114078000080FB00000F780093
:1015700002022000E00047001100110006003200C6
:10158000600047009000780069805000020032003F
:10159000D60A040000000000110020006800570077
:1015A00010884000B00A0400000000000000200085
:1015B000100798000000200020079800D2022000A9
:1015C000E00047001100110008003A00110020005F
:1015D0006400470010884000110020006800570098
:1015E00010884000040B040000000000B20220003C
:1015F000E00047001100110003003A001100200034
:101600006800570010884000CEB89700114078005D
:101610000080FB00000F780060004700901F7800FA
:101620001A0007002F00B1000000E0000D0032009A
:101630006202470094007800A00020000089B900F1
:10164000010320006000470010801000000A4100E4
:10165000110020006800570010884000040B0400AF
:10166000000000002E0090000000E00004003200A6
:101670006200470010007800600010000100370091
:101680001E0090000080FA00000006000000FA0032
:1016900092032000E80057001100110008003E00EE
:1016A00002032000E8005700110011000400390077
:1016B0001000200080407800640B0400000000004F
:1016C00000002000804078008180FB00010078004D
:1016D0000080FA00000006000800FA004EB99700EA
:1016E000124078000080FB00000F78000402200008
:1016F000600147001200120006003200600047003F
:10170000100178006900510002003200940B0400BF
:10171000000000001200200068005700100841007F
:101720006E0B04000000000000002000CF80DE00EF
:10173000100798002107980000002000300798004B
:101740004EB8970010427800D202200002405200AA
:1017500008003A001200200066004700100841000F
:10176000120020006800570010084100CA0B040056
:10177000000000004EB8970010427800B20220002E
:101780000240520003003A00120020006800570097
:10179000100841004EB99700124078000080FB000D
:1017A000000F780060004700901F7800B7FF070027
:1017B0002F00B1000000E000120032001E00900077
:1017C000AE009000A2002000030020002B2B070099
:1017D0000403200060014700120112000202780099
:1017E000CFA2DE00620147000419400005914800C5
:1017F000120020006800570010084100CA0B0400C6
:10180000000000003E0090000000E00006003200F2
:101810006200470030017800A001780060001100EC
:10182000E0801900020037001E009000AE0090001A
:101830000080FA00000006000000FA006A0157006C
:1018400062004100904078002003200001487800A9
:1018500012007800C00088009C05BA00B00080002B
:101860000080FA00000006000A00FA006A00570033
:1018700010007800100798004EB9970032007800E9
:10188000A20078002007980031079800000020008F
:10189000000F780060004700100278006C015700CC
:1018A0001200520015003D006400470040079800F8
:1018B000B01F7800A01F7800DFFF07004F00B100C5
:1018C0001E019000000978002200200062004700FD
:1018D0001008410022002000CF91DE004E00900051
:1018E00010184100109049001200200060004700CD
:1018F000100841004A0C0400000000006C00570072
:10190000100078004100DD004EB99700CF80DE0066
:1019100012194000129148000080FA0000000600F1
:101920004E00FA006000470021DC2E00050009008F
:10193000315878006600470081DC2E000500090060
:10194000315878006C004700E1DC2E0005000900EA
:10195000315878007200470041DD2E000400090074
:10196000315878007700470091DD2E00050009000E
:10197000315878007D004700F1DD2E000600090097
:1019800031587800400220000000470061DE2E0040
:10199000020009003158780000002000101F980054
:1019A00068005700901F78007A2207002F00B100CE
:1019B0006200500040179800610150006800570015
:1019C0001000410010427800A202200002405200A4
:1019D0000200320000002000D502370086022000FD
:1019E00006034700160078006100500068025700A7
:1019F0001401400000002000004978000400780035
:101A000010017800060078001000410010417800B5
:101A10000281FB00000320000001510052179800D2
:101A2000690051000400340072002000A002200070
:101A30000000470010081100A0022000000047002D
:101A4000100078004400DD00101F98008002200084
:101A50000000470010007800610140006800570056
:101A600010004100104178000281FB0000032000BB
:101A70000001510052179800690051000400340021
:101A800072002000A0022000000047001008110092
:101A9000A002200000004700100178002003200071
:101AA000000047001008410000002000406A880044
:101AB00000002000501798000000200040179800F8
:101AC00068005700100178008002200000004700E5
:101AD0001000410010417800604051000E003200BB
:101AE00068005700100078008402200004024700BC
:101AF00014004000104178000281FB00A002200089
:101B0000000047001008690010002000140A40007F
:101B1000600D0400000000002003200000004700CA
:101B200010027800A20220000201470012005200B9
:101B30000400320010002000406A880000002000ED
:101B40007B02370050002000801F7800680057009B
:101B5000901F780060004700801F780051FD07004B
:101B60006F00B10060015000D6003A0068025700D3
:101B7000542798001400780071004000104178004C
:101B800050D320000248780004007800901F7800AD
:101B900010002000801F780069FD07004F00B10091
:101BA000401798006601400068005700100141008E
:101BB00000002000004978005E20900010017800AD
:101BC00080022000000047004027980010004100DC
:101BD00064004000801F780077FD07002F00B100EF
:101BE000506A8800616A8800800220000000470077
:101BF00010007800640140006800570010014100A7
:101C000000002000004978005E209000100178005C
:101C10004E2090001000410062004000801F7800BC
:101C20004EFE07002F00B100706A8800800220007D
:101C30000000470010007800620140006800570073
:101C40001001410000002000004978005E20900053
:101C5000100178004E20900010004100801F780095
:101C60003EFE07002F00B100806A88006800570020
:101C7000901F780030002000801F780030FD0700A2
:101C80004F00B10040179800680157001200400053
:101C900062004000801F780047FD07002F00B10060
:101CA000201F9800311F980080022000000047008C
:101CB00010007800620140006800570010014100E8
:101CC00000002000004978005E209000100178009C
:101CD0004E20900010004100801F780036FD070064
:101CE0002F00B10020279800312798000200200023
:101CF000032724002E189000BE18900044290700E6
:101D00002E219000BE2190008B280700906A880049
:101D1000A16A880068005700901F780040002000EA
:101D2000801F780006FD07004F00B10068015700D2
:101D3000120040001041780060D520000248780071
:101D40005E209000901F780050002000801F7800D7
:101D5000FBFC07004F00B1004017980068015700D6
:101D60001200400063004000801F780012FD070051
:101D70002F00B100201F9800311F98008002200022
:101D80000000470010007800630140006800570021
:101D90001001410000002000004978005E20900002
:101DA000100178004E20900010004100801F780044
:101DB00001FD07002F00B10020279800312798006F
:101DC00002002000032724002E189000BE18900067
:101DD0000F2907002E219000BE21900056280700F1
:101DE000C06A8800D16A880068005700901F780098
:101DF00060002000801F7800D1FC07004F00B10078
:101E000068015700120040001041780070D5200092
:101E1000024878005E209000901F7800700020003B
:101E2000801F7800C6FC07004F00B1006801570012
:101E300012004000801F7800DFFC07002F00B10077
:101E400062E52000D3FE230066270700E06A8800D1
:101E5000F16A880068005700901F78008000200019
:101E6000801F7800B6FC07004F00B10068015700E2
:101E700012004000801F7800CFFC07002F00B10047
:101E8000006B8800116B880068005700901F780075
:101E900090002000801F7800A9FC07004F00B100CF
:101EA0006801570012004000801F78000AFE0700FA
:101EB0002F00B100206B8800316B880010002000DB
:101EC0009B01370050002000801F780068005700F9
:101ED000901F780066004700801F780071FC0700A3
:101EE0006F00B1006001500028003A006800570000
:101EF000901F780070002000801F780090FC070081
:101F00004F00B1006801570012004000801F7800A8
:101F100092FD07002F00B100406B88006800570059
:101F2000901F780080002000801F780084FC07004C
:101F30004F00B1006801570012004000801F780078
:101F40009DFC07002F00B100506B8800616B88007A
:101F500068005700901F780090002000801F7800D4
:101F600077FC07004F00B1006801570012004000E5
:101F7000801F780090FC07002F00B100706B880074
:101F8000816B88001000200069013700500020009C
:101F9000801F780068005700901F78006C00470091
:101FA000801F78003FFC07006F00B1006001500007
:101FB000CF003A0010002000906B880068005700A6
:101FC000901F780030002000801F78005CFC070024
:101FD0004F00B1006801570012004000801F7800D8
:101FE0005EFD07002F00B1005017980060015000FF
:101FF00004003D000000200050179800101004005D
:1020000000000000A002200000004700100178003E
:102010006C00510002003400C000200050179800EE
:10202000A002200000004700100078004017980030
:10203000A002200000004700100178006C00510051
:1020400016003D00A402200004024700140078009E
:102050004201DD0040D720000201400000002000C6
:102060000009780004007800100078004201DD00CB
:1020700040D7200002004000620140000000200024
:102080000009780012002000A00220000000470094
:1020900010084100181004000000000068005700FC
:1020A000901F780020002000801F780024FC07008B
:1020B0004F00B1006801570012004000801F7800F7
:1020C00026FD07002F00B100610150006217980043
:1020D0006300510084003D00C00220000000470062
:1020E000100078004201DD0080022000000047005F
:1020F00010011100421798006400510002003400E2
:102100004000200040179800000020005017980061
:10211000A002200000004700100278008202200088
:1021200002014700120052006F003D006800570096
:10213000901F7800A00220000000470010007800E7
:102140004200DD0064004000801F7800FCFB0700B7
:102150004F00B100101F98006801570012004000A6
:10216000104178006040510059003200680057006B
:1021700010017800200320000000470010004100FB
:1021800010427800C202200002405200500032008B
:10219000C00220000000470060279800100078006F
:1021A0004201DD00A00220000000470050279800F7
:1021B000100041004201DD0040D720000200400035
:1021C00040279800680057002027980010017800E9
:1021D000200320000000470010004100801F78000D
:1021E000DEFC07002F00B1004E21900000097800AE
:1021F0002E209000901F78005E2090001000780044
:102200004200DD006400400063004000801F780051
:10221000CBFB07004F00B100101F9800C202200046
:1022200002014700120178004212DD00A2022000E4
:1022300002014700120142004212DD0042D7200095
:102240000401410062014100222798006801570003
:1022500012004000801F7800C0FC07002F00B10072
:102260004101DD002E209000020878006E209000D1
:10227000100078004201DD005E2090001000410057
:102280004201DD0040D72000020040006202400011
:1022900032062000140011000D003600C00220009C
:1022A00000004700100078004201DD00A00220007D
:1022B00000004700100041004201DD0040D720002F
:1022C0000200400062014000300620000009780052
:1022D00012002000A002200000004700100841006A
:1022E000881004000000000010002000900037005B
:1022F00050002000801F780068005700901F780071
:1023000072004700801F780066FB07006F00B10075
:102310006001500006003A0077004700801F7800F7
:10232000B11507002F00B100100020008000370019
:1023300050002000801F780068005700901F780030
:102340007D004700801F780056FB07006F00B1003A
:102350006001500073003A0080C52F00F107200093
:10236000002798001127980010002000801F780097
:10237000A002200000004700801F78000004200019
:1023800000004700801F780037FD07006F00B10094
:1023900020002000801F7800E0022000000047009D
:1023A000801F78000004200000004700801F780094
:1023B0002DFD07006F00B100E00220000000470083
:1023C000B01F7800A01F780080DA2E00801F7800F0
:1023D00040DA2000801F7800681507008F00B100E8
:1023E00040DA2000801F78007F1507002F00B10021
:1023F0005E12900012002000A002200000004700A2
:1024000010081100600052003F003400000420005A
:102410000000470030027800A002780042FF2F0041
:10242000F30720000200520003805A0036003E00ED
:1024300020002000801F780080032000000047005B
:10244000801F78000004200000004700801F7800F3
:1024500005FD07006F00B10020002000801F7800FC
:10246000C003200000004700801F78000004200007
:1024700000004700801F7800FBFC07006F00B100E0
:1024800010002000801F780080022000000047001C
:10249000801F78000004200000004700801F7800A3
:1024A000F1FC07006F00B10080022000000047002F
:1024B000901F7800C003200000004700B01F780084
:1024C000A01F78008003200000004700B01F7800A4
:1024D000A01F780020DB2E00801F780040DA20004B
:1024E000801F780025150700EF00B10040DA2000BA
:1024F000801F78003C1507002F00B1000060FE002F
:10250000F811040000000000400220000000470015
:10251000801F7800341507002F00B1001000200044
:102520000300370020002000406A880000002000DF
:102530000080FA00000006000000FA00006F800032
:102540000000E0001100320068005700901F780082
:10255000901F07002F00B100810220000080500072
:10256000C180DE003062800068004000801F78007B
:10257000811F78005C0A07004F00B1006800570017
:10258000901F7800B31F07002F00B1000080FA00F1
:10259000000006001000FA0060004700B1DF2E00C6
:1025A0000C00090031587800506B8000616B80008E
:1025B0000200200003002000172607000000E000B2
:1025C00002003C0000002000010037001000200045
:1025D0000000E00058003200526B8000636B800006
:1025E000106F8000216F80000B2607000000E000C4
:1025F00002003D0000002000010037001000200014
:102600000000E0004C003200506B8000616B8000E5
:10261000106F8800216F8800326F800060005100C9
:1026200035003C00006F80000000E0000100320037
:1026300046120700C06A8000D16A8000406F88009F
:10264000516F8800906A8000A16A8000606F8800E6
:10265000716F8800706B8000816B8000806F8800D4
:10266000916F880060D5200010427800320520006C
:102670000240520005003A0002002000030028003A
:10268000C0DE2000101869001090690070D520008D
:1026900010427800720520000240520005003A0006
:1026A000020020000300280080DE200010186900CE
:1026B00010906900806A800000708800706A800055
:1026C00010708800506A8000616A8000F518070069
:1026D000207088001000200030708800000020006A
:1026E000801F7800281507002F00B1008D1F0700FC
:1026F0009813040000000000306F8000610050005B
:10270000306F8800801F780090DE2E00801F7800D8
:1027100040DA2000801F7800981407006F00B10095
:1027200040DA2000801F780083FF07002F00B100EF
:10273000EA13040000000000346F8000C2C02000D3
:10274000120052001F0032000000200070079800A5
:102750006E00470010017800760051000A003D002D
:1027600042DA20006E004700100141000002200004
:1027700000497800120020006E0047001008410058
:10278000A81304000000000042DA20006E00470099
:1027900010014100000020000049780040DA2000CC
:1027A000801F780064FF07002F00B1006060800088
:1027B000306F880060004700801F78005EFF0700D0
:1027C0002F00B1004060800051608000106F8800D1
:1027D000216F88000080FA00000006000800FA005F
:1027E0006A005700B01F7800A01F7800C5020700DC
:1027F0004F00B10000017800810178000000200046
:1028000001F82300C72507000000E00002003500A2
:102810000000200001003700100020000000E00050
:102820000300320000002000010020006D0037008E
:102830003EB89700CEB897003EB99700CEB9970042
:10284000E8240700200798003107980000002000C6
:1028500001F82300821F7800831F78002E0190006A
:10286000BE019000712507004F01BE00801F780057
:10287000811F78005D0007004F00B100000F780055
:10288000110798006A005700B01F7800A01F780059
:102890009C0207004F00B100000178008101780020
:1028A000F0282C0051F323005B2507000000E00016
:1028B00002003C0000002000010037001000200052
:1028C0000000E0000A0032001E0178009E01900026
:1028D0003EB89700CEB897004D260700801F7800BD
:1028E000811F7800A10207004F00B1003D003700B2
:1028F0006A01570032007800A20078000200200030
:1029000003002000872507000000E00002003500DA
:102910000000200001003700100020000000E0004F
:102920001D0032006000470030017800A0017800EF
:10293000000020000100280000006900818069007B
:102940003EB99700CEB9970031260700801F780066
:10295000811F7800850207004F00B1002007980012
:1029600031079800B0FD200091FC2300821F780001
:10297000831F78002E019000BE0190002B250700D8
:102980004F01BE0002002000030028000200680082
:1029900083806800130037003EB99700CEB99700D6
:1029A0001E0078009E00900019260700801F780006
:1029B000811F78006D0207004F00B10020079800CA
:1029C00031079800B0FD200091FC2300821F7800A1
:1029D000831F78002E019000BE0190001325070090
:1029E0004F01BE000080FA00000006000E00FA0051
:1029F0006A01570032007800A2007800020020002F
:102A000003002000472507000000E000020034001A
:102A10000000200001003700100020000000E0004E
:102A20000300320000002000010020006F0037008A
:102A30006A01570032007800A2007800000F780089
:102A4000110798000200780030017800A00178009A
:102A50000000200001F82300EF2407000000E00040
:102A600002003C00000020000100370010002000A0
:102A70000000E000070032001E0178009E01900077
:102A80000000200001F82300E1250700000F780076
:102A9000110798006A004700801F78006000470017
:102AA000B01F7800A01F7800520007006F00B1002F
:102AB000000F7800110798006A01470012017800A2
:102AC0004191DE00821F7800801F7800811F78000E
:102AD0009C0007006F00B100000F780011079800FC
:102AE0006A00570030017800A00178000000200043
:102AF00001F82300C82407000000E00002003C00A9
:102B00000000200001003700100020000000E0005D
:102B1000070032001E0178009E0190000000200096
:102B200001F82300BA250700000F7800110798006C
:102B300040012000400798001E0178009E0190008F
:102B40003EB89700CEB89700B12507006002470055
:102B50006407980034017800A4017800F624070087
:102B60000200200003002400A92507002007980088
:102B70003107980000027800810278006E00900012
:102B80000001780032007800A2007800040178008B
:102B900085017800E32407000000E0000200320015
:102BA0000000200001003700100020000000E000BD
:102BB00002003200F215040000000000640147002A
:102BC00032007800A2007800000F7800110798000A
:102BD000680047001000780061015000420798002B
:102BE000D5FF3A001E0078009E0090000080FA0099
:102BF000000006000400FA00600247006A01570066
:102C000032007800A2007800001A780001127800E3
:102C1000620042001001780000F827000000610007
:102C2000C701DE00E20720002EB89700028851009D
:102C3000E201420000F023001301680000F82700C1
:102C4000000061009309680034007800A400780057
:102C50000080FA00000006000600FA006A01570032
:102C600032007800A200780002002000030020005B
:102C7000AC2407000000E000020034000000200047
:102C800001003700100020000000E00003003200C7
:102C900000002000010020002800370060004700ED
:102CA000801F78006A005700B01F7800A01F7800CE
:102CB000D0FF07006F00B1000200200003002400D5
:102CC000C82307000200200003F823005724070050
:102CD00030BF9F0041BF9F001400200060014700EB
:102CE0001209120082002000821F780082E02E006C
:102CF000821F7800801F7800811F7800640607001B
:102D00008F00B100100798002107980030BF9F0086
:102D100041BF9F001E007800CF80DE000081EB00E5
:102D2000552307008221270013F32300AD2307005A
:102D30001E019000AE0190007F2407000080FA0081
:102D4000000006000400FA00E00147006A01570095
:102D500032007800A2007800801978008111780094
:102D6000628041001001780000F827000000610037
:102D70004701DE006C0057001001410022BF9F0098
:102D80006000510003003D00000020000100200011
:102D900023003700F30F20006C0157001280110050
:102DA000130034006A01570032007800A200780056
:102DB00002002000030020005A2407000000E00069
:102DC0000200350000002000010037001000200044
:102DD0000000E00003003200F0FF2F00F1F72F00A9
:102DE0000F003700F0FF2F00F1F727000C0037002D
:102DF00060004700E20140006C00570010007800BE
:102E00004700DD001301680000F8270000006100A2
:102E1000930968006001470032007800A200780042
:102E20000080FA00000006000800FA006A0157005E
:102E300032007800A2007800020020000300200089
:102E4000382407000000E0000200320000002000EB
:102E500001003700100020000000E00003003200F5
:102E60000000200001F823007B0037006A005700B3
:102E700030017800A0017800E04F2D00212B2400C4
:102E8000282407000000E0000200350000002000B8
:102E900001003700100020000000E00003003200B5
:102EA000F0FF2F00F1F727006B0037006A00570092
:102EB00030017800A001780000C52A00E12A2C002A
:102EC000D52307000000E00002003C0000002000C5
:102ED00001003700100020000000E0000300320075
:102EE00000002000010020005B0037006A0157004D
:102EF00032007800A20078000200200003002000C9
:102F0000082407000000E000020035000000200057
:102F10000100370010002000000F78000000E000E2
:102F20000500320002002000030028006A0057005C
:102F300010186900109069003EB89700CEB897004D
:102F4000B2A32A0083FB23002623070030BF9F0083
:102F500041BF9F00801F7800811F78007C0507001B
:102F60004F00B100CF16070030079800CF80DE0079
:102F70000081EB00C022070010079800210798008D
:102F80006A01570032007800A2007800821F7800A2
:102F9000831F78001E019000AE019000A32307005C
:102FA0004F01BE0030BF9F0041BF9F003E01900017
:102FB000821F780092002000821F7800C2E22E005B
:102FC000821F7800801F7800811F7800B0050700FD
:102FD0008F00B100801F7800811F780059FF070023
:102FE0006F00B10030BF9F0041BF9F001E007800FE
:102FF0000000E000160032006A005700300178003F
:10300000A0017800F0FF2F00F1F72700C52307008B
:103010000000E00002003200000020000100370044
:10302000100020000000E00003003200000020003B
:1030300001002000080037003EB99700CEB9970084
:103040000000200001F8230071240700020037006F
:103050003EB89700CEB897000080FA000000060046
:103060000000FA00020007009818040000000000A9
:103070000001BE00190007000470A70003F0A100C2
:1030800003F8A30013003A006509B10010003200F4
:10309000090035006928E100020035000100280020
:1030A0000000050000004000818048008502E90022
:1030B000FCFF3A0000000600F88F420005003500D2
:1030C0008100D1000080D3008502E800FCFF3A00B7
:1030D000000006008000EB0000000500C70ADE00CB
:1030E000F107B200F50FB20008003200E1CF420054
:1030F000020032000170A00024000500810F700062
:10310000010032000408050044000500810F700032
:1031100002003A00140005008502E90000004000AA
:1031200081C04800FCFF3B000170A00024000500A6
:103130000080FA00000006000600FA0000002000EF
:10314000000F78006A01570032007800A200780072
:103150000200200003002000722307000000E000AE
:1031600002003200000020000100370010002000A3
:103170000000E000030032000000200001002000F9
:103180005E0037006E01570032007800A200780020
:103190000200200003002000622307000000E0007E
:1031A0000200320000002000010037001000200063
:1031B0000000E000030032000000200001F82300BE
:1031C0004E0037006A01570032007800A2007800F4
:1031D0000200200003002000522307000000E0004E
:1031E0000200350000002000010037001000200020
:1031F0000000E000220032001EB89700AEB8970031
:1032000097FF070010079800210798000001EB00C6
:103210001922070000027800810278006E01570031
:1032200032007800A200780004017800850178005F
:103230003C2307000000E00002003A0000002000EC
:1032400001003700100020000000E0000300320001
:103250000000200001002000280037006200470025
:103260001001780060004700610861000200200042
:10327000030028006A0057001018690010906900C8
:103280006A005700B01F7800A01F780072FE070088
:103290004F00B10030BF9F0041BF9F001EB9970093
:1032A000AEB997004F22070030BF9F0041BF9F007B
:1032B000801F7800811F7800DBFE07004F00B100FF
:1032C00030BF9F0041BF9F001E0078000000E0005B
:1032D000080032006A00570030017800A001780031
:1032E00000002000010028000000690081806900C2
:1032F000020037003EB89700CEB897000080FA0071
:10330000000006000000FA006A0157003200780051
:10331000A200780002002000030020000123070023
:103320000000E0000200350000002000010037002E
:10333000100020000000E000080032006A00570082
:1033400030017800A0017800000020000100280072
:103350000000690081806900020037003EB89700D4
:10336000CEB897000080FA00000006000A00FA00BC
:103370006A005700B01F7800A01F7800E1FF070027
:103380004F00B100100798002107980002002000AC
:1033900003002000E32207000000E00002003200EA
:1033A0000000200001003700100020000000E000B5
:1033B0000300320000002000010020006B003700F5
:1033C0006200470030027800A00278000000200070
:1033D00001F823000401780085017800D12207005C
:1033E0000000E0000200350000002000010037006E
:1033F00010002000000F78000000E00007003200FD
:103400001E019000AE0190000000200001F8230092
:103410007F23070010079800210798001E009000E6
:10342000AE0090001E019000AE019000ED2107005B
:10343000300798004107980054002000841F78004E
:1034400044E52E00841F7800801F7800811F7800DB
:103450008F0407008F00B1001E019000AE019000A4
:10346000E021070010079800210798004000200085
:10347000801F7800C0E62E00801F7800660047009D
:10348000B01F7800A01F7800810407008F00B100F2
:1034900000017800810178001E009000AE009000CD
:1034A0005B23070010079800210798001E00780092
:1034B0000000E0000A003200B6FD200097FC230067
:1034C0006202470034017800A40178000600780009
:1034D0008700780055220700100798002107980000
:1034E0006A02570034007800A4007800020020002F
:1034F000030020008B2207000000E00002003500DE
:103500000000200001003700100020000000E00053
:103510000B0032006200470030027800A002780001
:10352000000020000100280000006A0081806A007D
:103530000003780081037800AA1A0400000000004C
:103540006202470034007800A4007800000378008D
:103550008103780006007800870078001007980043
:10356000210798001E009000AE0090000080FA0035
:10357000000006000000FA006E01570032007800DB
:10358000A200780002002000030020002222070091
:103590000000E00002003C000000200001003700B5
:1035A000100020000000E0000A0032001EB9970061
:1035B000AEB997003EB89700CEB897001423070025
:1035C000801F7800811F780068FF07004F00B1005E
:1035D0007D0037006A01570032007800A2007800B1
:1035E00002002000030020000B2207000000E00082
:1035F00002003D0000002000010037001000200004
:103600000000E0001A0032006E015700320078001E
:10361000A2007800020020000300200041220700E1
:103620000000E0000200350000002000010037002B
:10363000100020000000E0000D0032001EB99700CD
:10364000AEB997003EB89700CEB89700F0220700B9
:10365000801F7800811F780044FF07004F00B100F1
:10366000B2FD2000930424003322070056003700E7
:103670006A01570032007800A200780002002000A2
:1036800003002000272207000000E00002003500B0
:103690000000200001003700100020000000E000C2
:1036A0002A0032006E01570032007800A200780034
:1036B00002002000030020001A2207000000E000A2
:1036C000020035000000200001003700100020003B
:1036D0000000E0000D0032001EB99700AEB997005F
:1036E0003EB89700CEB89700C9220700801F780027
:1036F000811F78001DFF07004F00B100B2FD2000C0
:1037000093042C000C2207002F0037006E01570095
:1037100032007800A20078000200200003002000A0
:10372000002207000000E00002003200000020003C
:1037300001003700100020000000E000030032000C
:10374000B0FD200091FC2B001F0037006E015700D8
:1037500032007800A2007800020020000300200060
:10376000F02107000000E00002003200000020000D
:1037700001003700100020000000E00010003200BF
:103780006A01570032007800A20078000200200091
:1037900003002000A02107000000E00002003C0020
:1037A0000000200001003700100020000000E000B1
:1037B00003003200B0FD200091FC2300020037001E
:1037C00000002000010020000080FA000000060038
:1037D0001800FA00C06A8000D16A8000B2FD2000A3
:1037E00093042400FF20070002002000433324003C
:1037F00087220700000F780011079800906A800068
:10380000A16A8000B2FD200093042400F520070087
:1038100002002000433324007D2207004007980067
:103820005107980070D520001043780074052000DF
:103830000440530005003A00040020000500280061
:103840006000470010186A0010906A0060D52000E0
:1038500010437800340520000440530005003A006E
:1038600004002000050028006800470010186A00C6
:1038700010906A00C4002000680057001022B800B1
:1038800080DE200004024000040F9800340078001D
:10389000A4007800B2FD200093042400D12007008A
:1038A000020020004333240059220700200798001B
:1038B000310798000E089000640240003400780040
:1038C000A4007800B2FD200093042400C520070066
:1038D00002002000433324004D22070060079800B7
:1038E000710798000400200005002400841F780060
:1038F000851F78006803470036027800A60278002A
:1039000004017800850178004821070002002000AA
:10391000030024003E220700801F7800811F7800EA
:103920007F0307004F00B100801F7800811F7800DF
:1039300001FE07008F00B100200F9800310F9800A2
:1039400068004700B01F7800A01F7800110407002E
:103950004F00B100000F9800110F98006C00470055
:10396000B01F7800A01F78000A0407004F00B100C4
:103970000E0A90009E0A90000401780085017800EC
:1039800098200700000F9800110F980000002000F9
:1039900001002400801F7800811F78006400470028
:1039A00030037800A00378006002470034017800FB
:1039B000A401780006007800870078001B2107002A
:1039C000020020000300240011220700801F78005D
:1039D000811F7800520307004F00B100801F78005C
:1039E000811F7800D4FD07008F00B1000E0A9000FF
:1039F0009E0A900004017800850178007920070074
:103A00002E0A9000BE0A900004017800850178001B
:103A100049210700801F7800811F7800F3FB070011
:103A20004F00B100801F7800811F78006BFB0700FA
:103A30004F00B100020020000300240069200700AD
:103A4000020020004333240066200700B2FD20005E
:103A500093042400EE21070002002600A376240030
:103A60006020070062E52000D3FE23005D200700F0
:103A70004070880051708800040020000500240078
:103A8000841F7800851F7800801F7800811F7800D0
:103A9000A9FD07008F00B100000F9800110F9800DA
:103AA0000000200001002400801F7800811F7800A2
:103AB000100EF800120EF8009FFD07008F00B100F5
:103AC0000E0A90009E0A900004017800850178009B
:103AD00019210700801F7800811F7800C3FB0700B1
:103AE0004F00B10060708800717088006800470066
:103AF000B01F7800A01F7800A60307004F00B10098
:103B0000000F9800110F98006C004700B01F78005C
:103B1000A01F7800020307004F00B1000E0A9000BA
:103B20009E0A900004017800850178002D2007008E
:103B3000200F9800310F980068004700B01F7800F0
:103B4000A01F7800F60207004F00B100000F980098
:103B5000110F98006C004700B01F7800A01F78007C
:103B60008C0307004F00B1000E0A90009E0A9000DF
:103B700004017800850178001A200700000F9800E2
:103B8000110F98006400470030037800A00378000C
:103B90006002470034017800A40178000600780034
:103BA00087007800A1200700801F7800811F78001F
:103BB000780307004F00B1000E0A90009E0A9000A3
:103BC000040178008501780006200700000F9800A6
:103BD000110F98002E089000BE089000821F7800F8
:103BE000831F78000E0990009E0990008F20070027
:103BF0004F01BE00801F7800811F780064004700DD
:103C000030037800A0037800600247003401780098
:103C1000A401780006007800870078008320070060
:103C2000801F7800811F7800BD0207004F00B1009F
:103C3000000F9800110F98006C004700B01F78002B
:103C4000A01F7800530307004F00B1000E0A900038
:103C50009E0A90000401780085017800E11F0700AA
:103C6000801F7800811F780042FE07008F00B1009E
:103C70000200200043332400DA1F0700B2FD2000B9
:103C80009304240062210700A0708800B1708800AE
:103C90000200200003002000A22007000000E00036
:103CA0000200350000002000010037001000200055
:103CB0000000E00009003200A4708000B5708000B0
:103CC00000002000413B24000401780085017800B9
:103CD00099200700A0708800B17088000080FA0069
:103CE000000006002A00FA006000470001E82E00EC
:103CF00004000900315878006500470051E82E00A3
:103D00000E000900315878002603200084E12000CD
:103D10007400470014084300680057001002780040
:103D20006000520011003A00D07080000000E000F6
:103D30000C00320000002000D070880074004700A2
:103D4000901F7800700B2000801F7800EA010700A8
:103D50004F00B10060004700801F7800BD190700C8
:103D60002F00B100DE21040000000000D4708000AC
:103D70006000520010003A0010002000D07088004F
:103D800000002000F070880000002000E070880033
:103D900074004700901F7800700B2000801F78008F
:103DA000D50107004F00B10065004700801F780073
:103DB000A81907002F00B1003EB897000000E000EE
:103DC0005B01320074618000856180008270800038
:103DD00093708000040078008500780013200700AD
:103DE000300F9800410F980000027800810278009F
:103DF000B0618000C1618000040178008501780015
:103E0000482007000000E00002003500000020000C
:103E100001003700100020000000E0000600320022
:103E2000B0618000C1618000300F9800410F9800A0
:103E30003E1F0400000000007602470034007800B6
:103E4000A4007800020020000300200035200700B5
:103E50000000E000020035000000200001003700F3
:103E6000100020000000E0000400320000002000EC
:103E700001002000300F9800410F98003E0890008C
:103E8000CE089000D2608000E3608000551F0700DC
:103E9000700F9800011798000002780081027800E6
:103EA00090608000A16080000401780085017800A6
:103EB0001C2007000000E000020035000000200088
:103EC00001003700100020000000E0000600320072
:103ED00090608000A1608000700F9800011798002A
:103EE000AC1F04000000000094608000A56080000A
:103EF000000020000100280000036A0081836A009E
:103F00007E00470030027800A002780006007800AA
:103F1000870078000401780085017800BE1F070043
:103F20000000E00002003C0000002000010037001B
:103F3000100020000000E0000700320096608000C2
:103F4000A760800004002000050028007E004700D4
:103F500004186B0005906B00E46A8000F56A80002D
:103F60005061800061618000040178008501780063
:103F7000A91F07000000E00002003C000000200034
:103F800001003700100020000000E0000A003200AD
:103F90005261800063618000E06A8000F16A800005
:103FA0009B2007007E0990008E1190000D1F0700D6
:103FB000700F980001179800A4708000B570800001
:103FC000026B8000136B800004007800850078008D
:103FD000961F0700500F9800610F980000027800AC
:103FE00081027800000020004133240004017800A1
:103FF00085017800CB1F07000000E00002003500BB
:104000000000200001003700100020000000E00048
:104010000C0032007A00470030027800A0027800DD
:1040200002002000433B2400040078008500780053
:104030007E1F0700500F9800610F98005420040065
:10404000000000007A00470030027800A0027800EB
:104050000000200041332C00040178008501780025
:104060006D1F07000000E00002003C00000020007F
:1040700001003700100020000000E0000A003200BC
:104080007A00470030027800A0027800000020008B
:10409000413B24000401780085017800A61F070039
:1040A000500F9800610F98007A00470030027800A6
:1040B000A002780090618000A16180000401780076
:1040C00085017800971F07000000E000020035001E
:1040D0000000200001003700100020000000E00078
:1040E0000600320090618000A1618000500F9800AE
:1040F000610F9800B6200400000000009461800069
:10410000A5618000000020000100280000036A0073
:1041100081836A007A00470030027800A0027800AC
:104120000600780087007800040178008501780097
:10413000391F07000000E00002003C0000002000E2
:1041400001003700100020000000E00007003200EE
:1041500096618000A761800004002000050028000F
:104160007A00470004186B0005906B0002002000E5
:10417000433324005E089000EE08900024200700DE
:104180003261800043618000961E0700101798007E
:10419000211798000002780081027800F06080000A
:1041A0000161800004017800850178005D1F07002F
:1041B0000000E00002003500000020000100370090
:1041C000100020000000E00006003200F0608000D7
:1041D0000161800010179800211798002E2104001B
:1041E00000000000F46080000561800000002000F5
:1041F0000100280000036A0081836A002002200079
:104200000000470030027800A00278000600780025
:10421000870078000401780085017800FE1E070001
:104220000000E00002003C00000020000100370018
:10423000100020000000E00008003200F66080005E
:1042400007618000040020000500280020022000F3
:104250000000470004186B0005906B007E004700CB
:1042600030027800A0027800127180002371800073
:104270000400780085007800EC1E0700B260800022
:10428000C3608000571E07000612070000718800F7
:10429000C61220000602500004003400C0122000A4
:1042A0000071880062210400000000000671800097
:1042B00044ED2F000400530002003D0040ED2F00AC
:1042C00000718800200220000000470030027800C2
:1042D000A0027800427180005371800004007800D1
:1042E00085007800D11E07001261800023618000E4
:1042F0003C1E0700EB11070030718800C612200039
:104300000602500004003400C01220003071880002
:1043100098210400000000003671800044ED2F0059
:104320000400530002003D0040ED2F003071880072
:1043300004718000C0E12000301798001002520084
:1043400032002000110009000202D8003E12900045
:104350001400400040179800E0708800347180001D
:10436000E0E12000301798001002520032002000D7
:10437000110009000202D8003E1290001403400010
:10438000F6708800E4C320004E1090001484B90039
:1043900000C4200010B3B900E4D02000601D20004C
:1043A0001408140064D02000801D2000140843006D
:1043B00064D12000A01D2000140843000080FA00F2
:1043C000000006000E00FA0080C52F00F107200053
:1043D0004007980051079800C06A8000D16A8000A9
:1043E000000F780011079800906A8000A16A800091
:1043F000200798003107980060D52000104278000F
:10440000320520000240520005003A000200200060
:10441000030028006400470010186900109069002C
:1044200070D5200010427800720520000240520032
:1044300005003A0002002000030028006000470049
:1044400010186900109069008270800093708000DD
:10445000806F8000916F8000B71E070091110700E8
:104460006007980020002000801F7800600047004F
:10447000801F780068005700901F7800420E0700E8
:104480006F00B10020002000801F7800640047000A
:10449000801F780068005700901F78003A0E0700D0
:1044A0006F00B10010002000801F78006C004700F2
:1044B000801F780068005700901F7800320E0700B8
:1044C0006F00B1006A005700100078006007980084
:1044D00010002000801F78006C004700801F7800CB
:1044E00068004700801F7800270E07006F00B100AA
:1044F0000080FA00000006000000FA006A00570081
:10450000901F780068005700901F780040E92E0047
:10451000801F7800EA1707006F00B1000080FA00E2
:10452000000006000000FA006A005700901F7800A3
:1045300068005700901F780010EA2E00801F780056
:10454000DF1707006F00B1000080FA0000000600CE
:104550000600FA006A03570070012000CF80DE00D9
:1045600036027800A60278000000E900030035005A
:104570008502D1000482D300FBFF3700F00F20003A
:104580000002620024079800F00720000002520099
:10459000240798006000520013003D006A02570093
:1045A00034007800A40078000200200003002000FE
:1045B0005C1E07000000E000020035000000200043
:1045C00001003700100020000000E000030032006E
:1045D0000000200001F82B002B0037000000200015
:1045E0000100200028003700640047001002780016
:1045F00078005200030036003EB89700CEB897000E
:10460000210037003EB89700CEB89700251107006B
:104610000081EB00181D0700000F780011079800BB
:1046200000037800810378006A02570034007800A4
:10463000A40078000601780087017800391E070081
:104640000000E000020035000000200001003700FB
:10465000100020000000E000090032006000470068
:1046600030027800A00278000200200003F8230046
:104670000400780085007800EC1D07000200370078
:104680001E0078009E0090000080FA0000000600E6
:104690000400FA006E005700100078004201DD00AF
:1046A0006C0057001001410032007800A200780031
:1046B000000F7800110798001EB897000000E00076
:1046C000130032003EB89700CEB897001E01780064
:1046D0009E019000431D07006E01570012017800F3
:1046E0006101510012BF9F004212DD006C015700B2
:1046F0001202420034017800A40178000E1E070067
:10470000000F7800110798005C23040000000000EF
:104710001E0078009E0090000080FA000000060055
:104720000A00FA0000002000200798006A025700E3
:1047300034007800A400780002002000030020006C
:10474000F81D07000000E000020035000000200016
:1047500001003700100020000000E00007003200D8
:1047600004002000050028006A00570010186A00A5
:1047700010906A0010002000200798003EB89700B3
:10478000CEB8970032982F0023E22300151D0700B2
:1047900030BF9F0041BF9F00801F7800811F7800BD
:1047A0006BFF07004F00B1003007980041079800E9
:1047B0006A02570034007800A4007800821F780055
:1047C000831F78003E019000CE019000971D0700E6
:1047D0004F01BE000200200003082400011D070055
:1047E00030BF9F0041BF9F00000278008102780027
:1047F00000002000010024000401780085017800F9
:10480000C81D07000000E000020035000000200085
:1048100001003700100020000000E000110032000D
:104820006A00570030027800A002780002002000E1
:104830000300240004007800850078007B1D070039
:1048400030BF9F0041BF9F002E0090000000E0009D
:10485000020032000000200001003700100020009C
:10486000200798006A00570030027800A002780004
:104870000000200001F82300040178008501780081
:10488000A81D07000000E000020035000000200025
:1048900001003700100020000000E0000A00320094
:1048A00006002000070024006A0257003401780047
:1048B000A401780006007800870078005B1D0700DF
:1048C00030BF9F0041BF9F003EB89700CEB8970011
:1048D0003EB99700CEB99700C21C0700000F7800C0
:1048E0001107980044002000841F7800E4EA2E009D
:1048F000841F7800801F7800811F780064FF070004
:104900008F00B1003EB99700CEB99700B51C0700E3
:1049100030BF9F0041BF9F0030002000801F780003
:1049200020EC2E00801F780060004700B01F780048
:10493000A01F780056FF07008F00B100000178002B
:10494000810178003EB89700CEB89700301E07006E
:1049500030BF9F0041BF9F002E0090000000E0008C
:10496000080032006A00570030027800A002780088
:10497000000020000100280000006A0081806A0019
:10498000020037003EB89700CEB897000080FA00CA
:10499000000006000000FA006A00570030027800AC
:1049A000A0027800B0FD20009104240004017800EA
:1049B000850178005B1D07000000E0000200350063
:1049C0000000200001003700100020000000E0007F
:1049D0000D0032006A00570030027800A002780013
:1049E00042BE2C0063092400040078008500780092
:1049F0000E1D0700801F7800811F780048FF070008
:104A00004F00B1000C0037006A00570030027800F8
:104A1000A0027800B0FD200091FC23000401780082
:104A200085017800441D0700801F7800811F7800F1
:104A30003BFF07004F00B1000080FA0000000600B5
:104A40000600FA006000470021ED2E000500090075
:104A5000315878006E005700901F78006C005700A6
:104A6000901F78006A005700901F78006800570078
:104A7000901F7800070007008F00B100600047001A
:104A8000801F7800731607002F00B1000080FA0025
:104A9000000006000000FA00010920006A0057002B
:104AA00010804000801F7800010F20006800570030
:104AB00010804000801F780080ED2E00801F78005D
:104AC0007F1607006F00B100010920006E0057003B
:104AD00010804000801F7800010F20006C005700FC
:104AE00010804000801F780020EE2E00801F78008C
:104AF000731607006F00B1000080FA000000060086
:104B00000600FA0060004700C1EE2E000400090014
:104B1000315878006E005700901F78006C005700E5
:104B2000901F78006A005700901F780068005700B7
:104B3000901F7800D7FF07008F00B100600047008A
:104B4000801F7800431607002F00B1000080FA0094
:104B5000000006000800FA00F0628000CF80DE004E
:104B60000081EB00C41B0700B2FD20009304240069
:104B70001C1C07000200200043332400A41D070072
:104B8000801F7800811F7800E5FE07004F00B1000C
:104B90000200200083342C00121C0700200798001C
:104BA00031079800000178008101780000002000A2
:104BB000812C2400DB1C07000000E000020035000F
:104BC0000000200001003700100020000000E0007D
:104BD0000600320000002000812C240020079800ED
:104BE0003107980018260400000000006400470008
:104BF00030017800A001780000002000812C2C00FA
:104C0000851C07000000E00002003C0000002000BE
:104C100001003700100020000000E0000400320016
:104C200000002000812C2C002007980031079800FC
:104C3000E0628000CF80DE000081EB008E1B070069
:104C400002002000432B2400BB1C0700B2FD200003
:104C500093042400E31B07000200200043332400D8
:104C60006B1D0700801F7800811F7800ACFE0700D5
:104C70004F00B1002E019000BE019000D91B07002B
:104C8000880F070010079800E0628000CF80DE00E8
:104C90000081EB00781B070002002000432B24005A
:104CA000A51C0700B2FD200093042400CD1B0700C3
:104CB0000200200043332400551D0700801F7800A8
:104CC000811F780033FF07004F00B1002E019000D4
:104CD000BE019000C31B070002002000030824004F
:104CE000C01B07000200200003042400481D070029
:104CF0006C0F0700000F7800C4E220001401500080
:104D000007003A006200470010027800E2E220004B
:104D10001200520002003A00C02604000000000009
:104D20002E0EF8002C0EF80000002000801F7800E6
:104D300000002000801F780041FF07008F00B100B5
:104D4000600247001400780060718800620147002B
:104D5000120078007071880002007800901F7800BF
:104D600004007800901F780000002000801F780069
:104D700000002000801F780061FF07008F00B10055
:104D8000E0628000CF80DE000081EB003A1B07006C
:104D9000B2FD200093042400921B070002002000B3
:104DA000433324001A1D0700801F7800811F7800FC
:104DB0005BFE07004F00B10002002000032A240020
:104DC000881B0700370F070010079800E06280007B
:104DD000CF80DE000081EB00271B0700B2FD200022
:104DE000930424007F1B07000200200043332400AB
:104DF000071D0700801F7800811F7800E5FE07006F
:104E00004F00B10002002000032A2400751B070098
:104E10000200200003082400721B0700020020008B
:104E200003042400FA1C07001E0F0700000F78007F
:104E300004E320001401500007003A00620047001C
:104E40001002780022E320001200520002003A0013
:104E50007027040000000000360EF800340EF80041
:104E6000320EF800300EF800F5FE07008F00B1009A
:104E70006201470012007800E4E2200014044000C0
:104E800098718800E003470017007800C6E2200010
:104E900096024000857188000200780010007800BA
:104EA000600110000400780010024100B471880015
:104EB00007007800100078006001100006007800FC
:104EC00010004100A0718800841F7800801F7800C6
:104ED000881F7800851F780009FF07008F00B10048
:104EE0000080FA00000006000000FA006800570089
:104EF000901F78006A005700901F780010EF2E0076
:104F0000801F78006E1507006F00B1000080FA0066
:104F1000000006009A00FA006000470071172F0099
:104F2000040009003158780065004700C1172F00C0
:104F300004000900315878006A00470011182F005A
:104F400004000900315878006F00470061182F00F5
:104F5000040009003158780074004700B1182F0090
:104F60000C000900315878001002200000004700B2
:104F700081192F000B00090031587800D002200061
:104F800000004700411A2F00050009003158780041
:104F90003003200000004700A11A2F00050009007F
:104FA000315878009003200000004700011B2F00BB
:104FB0000500090031587800F00320000000470088
:104FC000611B2F00050009003158780050042000B3
:104FD00000004700C11B2F00050009003158780070
:104FE000B004200000004700211C2F00040009002D
:104FF000315878000005200000004700711C2F0088
:1050000004000900315878005005200000004700D6
:10501000C11C2F000500090031587800B0052000A0
:1050200000004700211D2F000500090031587800BD
:105030001006200000004700811D2F000400090019
:10504000315878006006200000004700D11D2F0075
:105050000200090031587800900620000000470047
:10506000011E2F000200090031587800C006200000
:1050700000004700311E2F0002000900315878005F
:10508000F006200000004700611E2F00020009000A
:10509000315878002007200000004700911E2F00A3
:1050A0000200090031587800500720000000470036
:1050B000C11E2F000200090031587800800720002F
:1050C00000004700F11E2F0002000900315878004F
:1050D000B007200000004700211F2F000200090038
:1050E00031587800E007200000004700511F2F00D2
:1050F0000400090031587800300820000000470003
:10510000A11F2F000300090031587800C0708000F3
:105110006B004000801F78009062800061004000BA
:10512000801F7800F4FC07004F00B100347080004D
:10513000600052000C003A00506A8000616A8000F2
:10514000580E0700801F78004E0DF800500DF80033
:10515000E0EF2E00801F7800D91407008F00B10007
:105160002E29040000000000506A8000616A80005F
:105170004C0E070044E020001402500044879800C1
:10518000706A800050879800806A8000608798006D
:105190006000520008003D00C40320008008200089
:1051A000000047001008420014002000A008200062
:1051B0000000470010081200A0082000000047006F
:1051C0001002780020E0200010025200548798005E
:1051D0006000520008003D00C4032000A008200029
:1051E000000047001008420014002000C008200002
:1051F0000000470010081200C0082000000047000F
:105200001002780000E0200010025200648798002D
:105210006000520004003D0084012000C00820000E
:1052200000004700100842008008200000004700EE
:10523000901F7800A008200000004700901F780011
:10524000C008200000004700901F780040F12E00A9
:10525000801F78009A1407008F00B100C070800092
:105260006B004000801F78007417200020C52000CC
:1052700010005200801F78009FFC07004F00B10013
:10528000106280000000E000080032005C0DF800B1
:105290005E0DF80060F22E00801F78008814070071
:1052A0006F00B1006C29040000000000E06A80007B
:1052B000F16A8000A2212100F3F12300491A0700BE
:1052C000801F7800811F780040F32E00801F780037
:1052D0007B1407006F00B1001471800025718000FD
:1052E000D0CC2C00C1E42B000401780085017800AB
:1052F0000C1B07000000E000020035000000200049
:1053000001003700100020000000E000180032000B
:105310001471800025718000D0CC2C00C1E42300E2
:105320000401780085017800BB1A07000000E00046
:1053300002003C00000020000100370010002000A7
:105340000000E0000A003200640920000402470067
:10535000000A2000004A7800740920000402470077
:10536000000C2000004A7800EC2904000000000036
:105370007409200004024700400C2000004A780015
:1053800010718000217180000200200003002000C5
:10539000A11A07000000E00002003C00000020000D
:1053A00001003700100020000000E000060032007D
:1053B000640920000402470020082000004A780009
:1053C000EC290400000000006409200004024700EA
:1053D00010082000004A78002060800031608000C2
:1053E0004270800053708000FE19070084708000B6
:1053F000957080000401780085017800861A070006
:105400000000E00002003C00000020000100370026
:10541000100020000000E000060032001004200010
:10542000801F7800361407002F00B1001C2A0400EA
:10543000000000003B140700C070800078004000AE
:10544000801F78007417200020C520001000520033
:10545000801F780028FC07004F00B1001062800018
:105460000000E00008003200100EF800120EF800F4
:1054700020F42E00801F7800111407006F00B10087
:105480005A2A0400000000008070800091708000A3
:1054900082942F0013052400D2190700801F780082
:1054A000811F7800E0F42E00801F780004140700AC
:1054B0006F00B10060092000000047001040780034
:1054C0000080FB00801F780070092000000047006A
:1054D000104078000080FB00801F7800B0F52E009F
:1054E000801F7800F61307006F00B1000D1407004D
:1054F000B06280000000E00014003A00C471800037
:10550000D5718000E0718000F171800004017800A5
:1055100085017800401A07000000E00002003C000E
:105520000000200001003700100020000000E00013
:105530000600320010042000801F7800F0130700DE
:105540002F00B100A82A040000000000F513070096
:10555000C070800078004000801F7800906280005A
:1055600061004000801F7800E3FB07004F00B1009E
:10557000380EF8003A0EF80040F62E00801F780032
:10558000CF1307006F00B100E6130700540220009C
:1055900080E1200010004200801F780090628000AF
:1055A00061004000801F7800D3FB07004F00B1006E
:1055B00036052000E4D22000140013003A00340025
:1055C00070698000CF80DE000081EB002A1907009F
:1055D0003232230033B5230082190700F4FD240082
:1055E000D5EC230004017800850178000F1A07002C
:1055F000D2CC2C00C3BC2300051B070004002000F4
:1056000005F0230004017800850178004A1A07009C
:10561000108F9800218F9800106280000000E00039
:105620000A0032002009200000004700B01F780067
:10563000A01F780000F72E00801F7800A01307003D
:105640006F00B1004C2B0400000000001E88900089
:10565000AE889000020020000311240061190700A9
:1056600002002000030A2400E91A070004002000B9
:105670000520240004017800850178002E1A070017
:10568000801F7800811F7800F0F72E00801F7800BF
:105690008B1307006F00B10010002000007288001B
:1056A000662B040000000000007280000000E00093
:1056B00006003200E0F82E00801F780080130700FB
:1056C0002F00B10000002000007288009513070031
:1056D0000403200060C4200010A2B900000D2000C7
:1056E0000403400084E12000E0082000000047009F
:1056F0001408530094628000000920000000470055
:1057000061084200147280002572800000002000B1
:10571000010A24000401780085017800011A0700BD
:105720000000E0000200350000002000010037000A
:10573000100020000000E0005B003200E0082000C4
:1057400000004700901F780000092000000047007B
:10575000901F780068FB07004F00B10014728000B2
:105760002572800030728000417280000401780050
:1057700085017800A81907000000E00002003C0045
:105780000000200001003700100020000000E000B1
:105790000600320010042000801F78005813070014
:1057A0002F00B100D82B0400000000005D1307009B
:1057B000420EF800440EF80070F92E00801F7800A9
:1057C0003F1307006F00B100E00820000000470011
:1057D000100078006D004000801F78000009200054
:1057E00000004700901F780043FB07004F00B10006
:1057F0004A0EF8004C0EF80000FB2E00801F7800C7
:105800002F1307006F00B100E008200000004700E0
:10581000100078007A004000801F78000009200006
:1058200000004700901F780033FB07004F00B100D5
:105830007472800085728000D0618000E161800018
:105840000401780085017800B61907000000E00027
:105850000200350000002000010037001000200089
:105860000000E0000600320010042000801F7800D5
:10587000231307002F00B100422C04000000000099
:10588000281307004E0EF800500EF800C0FB2E0043
:10589000801F78000A1307006F00B1002113070072
:1058A000A42C040000000000E008200000004700D5
:1058B000901F78000009200000004700901F78002A
:1058C0000DFB07004F00B10060004700801F78000B
:1058D000E01207002F00B100E008200000004700A0
:1058E000100078006D004000801F78000009200043
:1058F00000004700901F7800FFFA07004F00B1003A
:1059000065004700801F7800D21207002F00B10009
:10591000E008200000004700100078007A004000F6
:10592000801F78000009200000004700901F7800C9
:10593000F1FA07004F00B1006A004700801F7800AD
:10594000C41207002F00B1003470800060005200C4
:10595000D40132000403200060C4200010A2B9006A
:10596000D00D20000402400080E120001000520011
:1059700070879800801F78003418200020C5200010
:1059800010005200801F7800DBFA07004F00B100C2
:1059900044708000557080007060800081608000DD
:1059A00004017800850178001B1907000000E00061
:1059B00002003C0000002000010037001000200021
:1059C0000000E0003E003200106280000000E000B5
:1059D00008003200080EF8000A0EF80090FC2E00B5
:1059E000801F7800B61207006F00B1005C2D040024
:1059F000000000004070800051708000A221210052
:105A0000F3F123007718070002002400C36124008B
:105A1000FF190700000278008102780000002000D2
:105A200001F8230004017800850178003D19070082
:105A30000000E000020035000000200001003700F7
:105A4000100020000000E0001000320040708000D4
:105A500051708000A2212100F3F12300611807009A
:105A600002002000A3472400E9190700801F7800E6
:105A7000811F780040FD2E00801F780090120700E3
:105A80006F00B1005C2D0400000000004070800039
:105A90005170800082942F001305240051180700D4
:105AA000801F7800811F780010FE2E00801F780074
:105AB000831207006F00B100682D04000000000091
:105AC0006F004700801F7800621207002F00B100AE
:105AD000E008200000004700100078006D00400042
:105AE000801F7800B416200020C52000100052004E
:105AF000801F780080FA07004F00B1007400470053
:105B0000801F7800531207002F00B10064708000DE
:105B100075708000006080001160800004017800D2
:105B200085017800FF1807000000E0000200350042
:105B30000000200001003700100020000000E000FD
:105B40000600320010042000801F78006C1207004D
:105B50002F00B100B02D04000000000071120700FA
:105B6000106280000000E000080032000C0EF80017
:105B70000E0EF800D0FE2E00801F78005012070095
:105B80006F00B100282E040000000000607080004B
:105B900071708000A2212100F3F123001118070089
:105BA00002002400C3612400991907000002780054
:105BB000810278000000200001F823000401780031
:105BC00085017800D71807000000E00002003500CA
:105BD0000000200001003700100020000000E0005D
:105BE000100032006070800071708000A2212100DE
:105BF000F3F12300FB17070002002000A347240055
:105C000083190700801F7800811F780080FF2E0015
:105C1000801F78002A1207006F00B100282E0400B0
:105C200000000000607080007170800082942F007E
:105C300013052400EB170700801F7800811F7800F0
:105C400050002F00801F78001D1207006F00B10068
:105C5000341207000403200060C4200010A2B90021
:105C6000F00820000403400084E12000E008200048
:105C700000004700140853003615200024C52000FA
:105C8000000920000000470014085300E46A800067
:105C9000F56A80000000200001F023000401780074
:105CA000850178005C1807000000E00002003C005D
:105CB0000000200001003700100020000000E0007C
:105CC000A8003200E008200000004700901F780084
:105CD000840220000009200000004700100042005C
:105CE000801F78000FFA07004F00B100100220005B
:105CF00000004700801F7800D61107002F00B10078
:105D0000106280000000E00032003200E008200055
:105D100000004700100078006D004000801F7800F0
:105D20000009200000004700901F7800F2F90700EA
:105D30004F00B100520EF800540EF80010012F0071
:105D4000801F7800DE1107006F00B100E00820001E
:105D500000004700100078007A004000801F7800A3
:105D60000009200000004700901F7800E2F90700BA
:105D70004F00B100560EF800580EF800D0022F0068
:105D8000801F7800CE1107006F00B1007402200060
:105D9000E00820000000470010004200801F78004B
:105DA0000009200000004700901F7800D2F907008A
:105DB0004F00B1005A0EF8005C0EF80070042F007E
:105DC000801F7800BE1107006F00B1006E2F040025
:105DD00000000000E00820000000470010007800EC
:105DE0006D004000801F780000092000000047007F
:105DF000901F7800C0F907004F00B100907280003A
:105E0000A1728000A2212100F3F123007517070081
:105E1000801F7800811F780000062F00801F780007
:105E2000A71107006F00B100E00820000000470044
:105E3000100078007A004000801F780000092000E0
:105E400000004700901F7800ABF907004F00B10039
:105E5000B0728000C172800082942F00130524006C
:105E600060170700801F7800811F7800C0072F008F
:105E7000801F7800921107006F00B10074022000AB
:105E8000E00820000000470010004200801F78005A
:105E90000009200000004700901F780096F90700D5
:105EA0004F00B100D0728000E1728000A221210079
:105EB000F3F123004B17070002002000A347240042
:105EC000D3180700801F7800811F780070092F0009
:105ED000801F78007A1107006F00B10014728000F3
:105EE000257280000000200001F8230004017800E2
:105EF000850178000B1807000000E0000200350063
:105F00000000200001003700100020000000E00029
:105F10001000320044032000E00820000000470089
:105F200010004200801F7800000920000000470098
:105F3000901F780070F907004F00B1005E0EF80066
:105F4000600EF800200B2F00801F78005C11070006
:105F50006F00B10010002000107388005230040060
:105F60000000000014738000610052004D003A00F0
:105F7000E008200000004700901F78008402200005
:105F8000000920000000470010004200801F780038
:105F900064F907004F00B100D00220000000470064
:105FA000801F78002B1107002F00B100E0082000AF
:105FB00000004700100078006D004000801F78004E
:105FC0000009200000004700901F78004AF90700F0
:105FD0004F00B1003003200000004700801F780010
:105FE0001C1107002F00B100E0082000000047004E
:105FF000100078007A004000801F7800000920001F
:1060000000004700901F78003BF907004F00B100E7
:106010009003200000004700801F78000D1107004A
:106020002F00B10074022000E008200000004700AB
:1060300010004200801F7800000920000000470087
:10604000901F78002CF907004F00B100F0032000EA
:1060500000004700801F7800FE1007002F00B100ED
:1060600044032000E0082000000047001000420028
:10607000801F78000009200000004700901F780072
:106080001DF907004F00B100500420000000470038
:10609000801F7800EF1007002F00B10000002000E3
:1060A00010738800347080006000520016003200C7
:1060B000206080003160800042708000537080005A
:1060C000C816070084708000957080000401780075
:1060D00085017800501707000000E00002003C0036
:1060E0000000200001003700100020000000E00048
:1060F00005003A006468800060005200020032002F
:10610000423104000000000054688000600052002A
:106110005C003A00C07080006B004000801F780077
:1061200080072000801F7800F3F807004F00B100BF
:10613000446B80006300520007003D00680DF800CA
:10614000C00C2F00801F7800DD1007004F00B10049
:10615000B630040000000000680DF800300E2F007B
:10616000801F7800D61007004F00B100C07080007B
:106170006B004000801F7800600E2000801F7800B8
:10618000DDF807004F00B10060D520001040780016
:106190000080FB00801F7800520DF800540DF800BD
:1061A000000F2F00801F7800C51007008F00B1007E
:1061B000C070800078004000801F7800600E2000D2
:1061C000801F7800CCF807004F00B10070D5200088
:1061D000104078000080FB00801F7800580DF80008
:1061E0005A0DF800E00F2F00801F7800B410070050
:1061F0008F00B100C070800078004000801F7800E0
:10620000E0062000801F7800BBF807004F00B100B7
:10621000506B8000616B80000200200003002000B2
:10622000FD1607000000E00002003C000000200016
:1062300001003700100020000000E00008003200DC
:106240006A0DF8006C0DF800C0102F00801F780058
:106250009B1007006F00B1003A31040000000000FD
:10626000B004200000004700801F7800791007006C
:106270002F00B1001000200020738800AC31040012
:1062800000000000247380006100520032003A00D8
:10629000C07080006B004000801F780080072000E5
:1062A000801F780094F807004F00B100000520001F
:1062B00000004700801F7800661007002F00B10023
:1062C000C07080006B004000801F7800600E2000CE
:1062D000801F780088F807004F00B10050052000AB
:1062E00000004700801F78005A1007002F00B100FF
:1062F000C070800078004000801F7800600E200091
:10630000801F78007CF807004F00B100B005200026
:1063100000004700801F78004E1007002F00B100DA
:10632000C070800078004000801F7800E0062000E8
:10633000801F780070F807004F00B10010062000A1
:1063400000004700801F7800421007002F00B100B6
:106350000000200020738800000020004087980083
:106360000403200060C4200010A2B900900D20009A
:106370000403400084E12000E00820000000470002
:1063800014085300C0082000008F9800006B8000A4
:10639000116B8000C309070060879800C4062000C5
:1063A00004025000648798006000520004003D0021
:1063B00084162000C008200000004700100842009A
:1063C000C008200000004700100278006200200092
:1063D000110009000202D8006087980064002000C4
:1063E0000480B900608798007602200084082000AD
:1063F000040247001400130090003D00C008200074
:10640000000047001000780066034000668798008F
:106410008416200004005300040035008416200078
:10642000C00820000000470010081200C00820002B
:106430000000470010027800E2012000110009006E
:106440000202D80001007800600250000A00320009
:1064500040DA2000860820000603470016024000AC
:10646000D0022000004A780010002000160B4000E7
:106470001A33040000000000A4052000C00820001A
:106480000000470010007800110009000400D80047
:10649000010078006002500012003200C0082000A5
:1064A00000004700901F780010122F00801F780016
:1064B00044DA20008008200000004700100042005D
:1064C000801F78002D0507006F00B1003400200008
:1064D000800820000000470010084200123304002A
:1064E0000000000040DA2000860820000603470074
:1064F00016024000D0022000004A78001000200060
:10650000160B4000C23204000000000064092000A5
:1065100004024700E0042000004A7800F032040042
:10652000000000006409200004024700500420001D
:10653000004A7800F03204000000000064092000E6
:106540000402470030052000004A7800F0320400C1
:1065500000000000640920000402470070052000CC
:10656000004A7800F03204000000000064092000B6
:1065700004024700F0032000004A7800F0320400D3
:1065800000000000C0082000000047001002780052
:1065900060005200DDFF3200A6052000C408200084
:1065A0000402470014001300DEFF3200460B2000F7
:1065B000C40820000402470014001300DFFF32006B
:1065C000C00820000000470010037800E4102000FD
:1065D00004005300DFFF3200B63204000000000068
:1065E00040DA20008608200006034700160240001B
:1065F0006009200000004700104A7800060078007B
:1066000010007800610240004487980040DA2000C2
:1066100004024000D0022000004A78001000200050
:10662000160B4000C4002000C008200000004700F6
:1066300010084200F43104000000000044DA200099
:1066400080082000000047001002420000002000E7
:10665000004A7800006B8000116B80001109070070
:106660004087980064002000110009000400D80051
:1066700001007800408798006002500005003A0051
:1066800064DC200000002000004A78005033040041
:106690000000000074DC200000002000004A7800A8
:1066A0000009200000004700100278008008200048
:1066B00000004700100352004687980074DC200059
:1066C00000002000004A7800E00820000000470099
:1066D000100078006A004000801F7800861F780054
:1066E00090F707004F00B10070DA2000801F78009B
:1066F00060122F00801F7800710F07004F00B1005B
:10670000A4708000B5708000026B8000136B800065
:106710000400780085007800C4150700E108070030
:1067200060879800E008200000004700901F780074
:10673000A4052000000920000000470010004200CE
:10674000801F780077F707004F00B100C0082000D5
:106750000000470010027800600052000B003A0071
:10676000307080000000E00008003200600DF8008A
:10677000620DF800B0122F00801F7800500F070044
:106780006F00B100D233040000000000600DF8007B
:10679000620DF80070132F00801F7800480F07006B
:1067A0006F00B1005F0F0700307080000000E00054
:1067B00024013200A06280000000E00001003200ED
:1067C000E4F80700C008200000004700100378002C
:1067D000C4F42F000400530006003D00841620007E
:1067E000C008200000004700100842000C340400DC
:1067F00000000000460B2000C408200004024700EF
:10680000140013000400340084162000C008200087
:106810000000470010081200000020005087980078
:10682000A008200000004700100278007F005200FE
:106830000C003D0044DA2000A008200000004700C2
:106840001002420000022000004A780014002000DC
:10685000A008200000004700100842001034040087
:106860000000000044DA2000A008200000004700DB
:106870001002420000002000004A780006FA2F00B3
:10688000C408200004024700140013002400340050
:1068900006062000C408200004024700140013006C
:1068A0001F003D00A4052000C00820000000470094
:1068B00010024200448F9800548798006200200024
:1068C000110009000202D8000100780040879800FA
:1068D000640020004E889000110009000400D800D8
:1068E00050879800600250000B003500A00820007F
:1068F00000004700100278007F00520006003D00B3
:1069000044DA2000A00820000000470010024200E6
:1069100080042000004A7800943404000000000045
:1069200000002000408798008008200000004700F9
:106930001002780000092000000047001002420009
:1069400044879800E008200000004700100078000D
:1069500074004000801F7800841F7800F1F6070063
:106960004F00B100C008200000004700100278006E
:106970006000520008003A0040DA2000801F7800D2
:10698000E0132F00801F7800CD0E07004F00B100EC
:106990000035040000000000C0082000000047008F
:1069A00010027800670052000700350096FF2F00A4
:1069B000C4082000040247001400130002003C0039
:1069C000F43404000000000040DA2000801F78004A
:1069D000D0142F00801F7800B90E07004F00B100BF
:1069E000003504000000000040DA2000801F78001D
:1069F00020152F00801F7800B10E07004F00B10056
:106A0000C00820000000470010027800600052001B
:106A100024003A00E0082000000047001000780041
:106A20006A004000801F7800000920000000470035
:106A30001000780067005000801F7800AEF6070055
:106A40004F00B1006006200000004700801F780062
:106A5000800E07002F00B100E00820000000470072
:106A6000100078006A004000801F7800F40B2000BE
:106A7000000920000000470010004200801F78003D
:106A80009DF607004F00B10090062000000047006F
:106A9000801F78006F0E07002F00B1001E36040023
:106AA00000000000C008200000004700100278002D
:106AB000600052002E003D00E0082000000047006A
:106AC000100078006A004000801F78000009200054
:106AD000000047001000780067005000801F780019
:106AE00085F607004F00B10066FA2F00C4082000A9
:106AF000040247001400130007003D00C0062000F8
:106B000000004700801F7800520E07002F00B100E0
:106B10009635040000000000F00620000000470049
:106B2000801F78004B0E07002F00B100E008200006
:106B300000004700100078006A004000801F7800C5
:106B4000F40B200000092000000047001000420064
:106B5000801F780068F607004F00B1002007200072
:106B600000004700801F78003A0E07002F00B10098
:106B7000C0082000000047001002780060005200AA
:106B80002E003400E00820000000470010007800CC
:106B90006A004000801F7800F40B200000092000EC
:106BA0000000470010004200801F780052F60700E6
:106BB0004F00B100A6052000C408200004024700D1
:106BC00014001300070034005007200000004700A5
:106BD000801F78001F0E07002F00B100FC35040055
:106BE000000000008007200000004700801F7800A0
:106BF000180E07002F00B100E00820000000470039
:106C0000100078006A004000801F78000009200012
:106C1000000047001000780067005000801F7800D7
:106C200035F607004F00B100B00720000000470014
:106C3000801F7800070E07002F00B100A237040064
:106C400000000000906B80000000E000BD003200FA
:106C5000306280006B0240007487980000002000C2
:106C6000906B8800841F7800B0002000801F78009F
:106C70009DF807004F00B1000000200040879800F9
:106C80008008200000004700100278006C005200CD
:106C900038003D0080082000000047001000780008
:106CA0004202DD0040D720000400400062034000A3
:106CB0002403200016001200060031007409200091
:106CC0000402470000092000004A78009C360400B6
:106CD000000000008008200000004700100078003D
:106CE0004202DD0040D72000040040006202400064
:106CF000100320001402100072002000110009008F
:106D00000282D8000409200000024200700920001D
:106D1000000047000448780004437800640920001C
:106D200004405300040036007409200004024700A8
:106D300060092000004A7800700920000000470028
:106D4000104078000080FB00801F780070152F0035
:106D5000801F7800DA0D07004F00B10014002000FA
:106D60008008200000004700100842004036040060
:106D700000000000E008200000004700100078003C
:106D800061004000801F7800B0002000801F780064
:106D900055F807004F00B100000020004087980020
:106DA0008008200000004700100278006C005200AC
:106DB0002E003D00800820000000470010007800F1
:106DC0004202DD0040D72000040040006203400082
:106DD0001403200016001200060039007409200078
:106DE0000402470060092000004A780018370400B8
:106DF000000000008008200000004700100078001C
:106E00004202DD0040D72000040040006200400044
:106E10001002780072002000110009000282D800E0
:106E2000060920007409200004024700004A4300BC
:106E30007009200000004700104078000080FB002F
:106E4000801F780040162F00801F78009C0D0700DF
:106E50004F00B1001400200080082000000047000F
:106E600010084200D036040000000000E0082000B6
:106E7000000047001000780062004000801F78008A
:106E8000B0002000801F780017F807004F00B10005
:106E9000E007200000004700801F78006D0D07000C
:106EA0002F00B100000020004087980080082000DB
:106EB00000004700100278006C00520021003D00E5
:106EC0008008200000004700100078004202DD002A
:106ED00040D72000040040001002780060005200FB
:106EE0000D003200800820000000470010007800EC
:106EF0004202DD0040D7200004004000901F7800CF
:106F000010172F00801F78006D0D07004F00B10093
:106F10009637040000000000300820000000470001
:106F2000801F78004B0D07002F00B10014002000D7
:106F30008008200000004700100842005637040077
:106F4000000000000080FA00000006000600FA00C1
:106F500060004700E11F2F0004000900315878004D
:106F600060004700801F78003A0D07002F00B10035
:106F70000080FA00000006000600FA0080012000F0
:106F8000000F780032628000300020000090B900CD
:106F9000F0014000230798006801570012007800B4
:106FA000100798001280110007003400C00D200067
:106FB000000F780064004700100078006101400075
:106FC00062004700100811006200470010017800BD
:106FD000D00020000090B900100798007A0040000F
:106FE00010079800801F780060004700901F78000D
:106FF00030202F00801F7800310D07006F00B10096
:107000000080FA00000006004A00FA006000470015
:10701000514A2F00030009003158780064004700EE
:10702000914A2F000300090031587800680047009A
:10703000D14A2F0003000900315878006C00470046
:10704000114B2F00030009003158780070004700F1
:10705000514B2F0006000900315878007700470097
:10706000C14B2F00080009003158780000022000B1
:1070700000004700514C2F000300090031587800F0
:107080004002200000004700914C2F00040009003E
:10709000315878009002200000004700E14C2F009A
:1070A0000300090031587800D0022000000047009A
:1070B000214D2F00050009003158780030032000D1
:1070C00000004700814D2F0003000900315878006F
:1070D0007003200000004700C14D2F00030009008D
:1070E00031587800B003200000004700014E2F0007
:1070F0000200090031587800E0032000000047003A
:10710000314E2F000400090031587800300420006F
:1071100000004700814E2F0001000900315878001F
:107120005004200000004700A14E2F000400090079
:107130003158780068005700901F78008EFF0700D4
:107140002F00B100680057001001780061E62000B0
:107150001100510006003A00A0042000801F7800B2
:10716000E70C07002F00B100BA380400000000004F
:10717000EC0C0700A23B040000000000000CF8002B
:10718000020CF80000212F00801F780040DA200058
:10719000801F7800F90107008F00B1008E3C0400C9
:1071A00000000000040CF800060CF80080222F00FC
:1071B000801F780040DA2000801F7800EF01070070
:1071C0008F00B1008E3C040000000000080CF800A5
:1071D0000A0CF80000242F00801F780040DA2000FD
:1071E000801F7800E50107008F00B1008E3C04008D
:1071F000000000000C0CF80080252F00801F780094
:1072000040DA2000801F7800DC0107006F00B10029
:107210008E3C0400000000000E0CF800100CF8007A
:10722000E0262F00801F780040DA2000801F7800C1
:10723000D20107008F00B1008E3C04000000000066
:10724000120CF800140CF80060282F00801F780042
:1072500040DA2000801F7800C80107008F00B100CD
:107260008E3C040000000000160CF800180CF8001A
:10727000E0292F00801F780040DA2000801F78006E
:10728000BE0107008F00B1008E3C0400000000002A
:107290001A0CF8001C0CF800602B2F00801F7800DF
:1072A00040DA2000801F7800B40107008F00B10091
:1072B0008E3C0400000000001E0CF800200CF800BA
:1072C000E02C2F00801F780040DA2000801F78001B
:1072D000AA0107008F00B1008E3C040000000000EE
:1072E000220CF800240CF800602E2F00801F78007C
:1072F00040DA2000801F7800A00107008F00B10055
:107300008E3C040000000000260CF800280CF80059
:10731000E02F2F00801F780040DA2000801F7800C7
:10732000960107008F00B1008E3C040000000000B1
:107330002A0CF8002C0CF80060312F00801F780018
:1073400040DA2000801F78008C0107008F00B10018
:107350008E3C0400000000002E0CF800300CF800F9
:10736000E0322F00801F780040DA2000801F780074
:10737000820107008F00B1008E3C04000000000075
:10738000360CF800380CF80060342F00801F7800AD
:1073900040DA2000801F7800780107008F00B100DC
:1073A0008E3C040000000000320CF800340CF800A1
:1073B000E0352F00801F780040DA2000801F780021
:1073C0006E0107008F00B1008E3C04000000000039
:1073D0003A0CF8003C0CF80060372F00801F780052
:1073E00040DA2000801F7800640107008F00B100A0
:1073F0008E3C040000000000F161800061805000BC
:1074000004003A0060004700800078000E3A040053
:107410000000000064004700800078000100780050
:10742000801F7800E0382F00801F780040DA2000AD
:10743000801F7800510107006F00B1008E3C0400EE
:1074400000000000016280006180500004003A00EA
:107450006800470080007800343A04000000000013
:107460006C0047008000780001007800801F7800E1
:10747000403A2F00801F780040DA2000801F7800FB
:107480003E0107006F00B1008E3C040000000000C8
:10749000106280000000E00004003200700047002D
:1074A000800078005A3A040000000000770047008E
:1074B0008000780001007800801F7800A03B2F003A
:1074C000801F780040DA2000801F78002B01070021
:1074D0006F00B1008E3C040000000000440CF80076
:1074E000D03C2F00801F780040DA2000801F7800F9
:1074F000220107006F00B1008E3C04000000000074
:10750000306280000000E000050032000002200030
:107510000000470080007800963A04000000000058
:107520004002200000004700800078000100780041
:10753000801F7800303E2F00801F780040DA200046
:10754000801F78000D0107006F00B1008E3C040021
:1075500000000000480CF800603F2F00801F7800FA
:1075600040DA2000801F7800040107006F00B1009E
:107570008E3C040000000000307080000000E0003D
:1075800005003200900220000000470080007800D3
:10759000D23A040000000000D002200000004700A2
:1075A0008000780001007800801F7800C0402F0024
:1075B000801F780040DA2000801F7800EF0007006D
:1075C0006F00B1008E3C0400000000004A0CF8007F
:1075D0004C0CF800F0412F00801F780040DA2000AA
:1075E000801F7800E50007008F00B1008E3C04008A
:1075F000000000004E0CF800500CF80050432F0023
:10760000801F780040DA2000801F7800DB00070030
:107610008F00B1008E3C040000000000520CF80006
:10762000D0442F00801F780040DA2000801F7800AF
:10763000D20007006F00B1008E3C04000000000083
:10764000B06280000000E00005003200300320003E
:107650000000470080007800363B04000000000076
:1076600070032000000047008000780001007800CF
:10767000801F780030462F00801F780040DA2000FD
:10768000801F7800BD0007006F00B1008E3C040031
:1076900000000000A06280000000E0000500320051
:1076A000B00320000000470080007800603B040029
:1076B00000000000E0032000000047008000780088
:1076C00001007800801F780090472F00801F78000D
:1076D00040DA2000801F7800A80007006F00B1008A
:1076E0008E3C040000000000407380000000E000B9
:1076F00005003200300420000000470080007800C0
:107700008A3B0400000000005004200000004700F5
:107710008000780001007800801F7800F0482F007A
:10772000801F780040DA2000801F78009300070057
:107730006F00B1008E3C0400000000008E3C04008D
:107740000000000068005700900078006080500042
:107750008AFE320068005700900078006180500077
:1077600090FE320068005700900078006280500060
:1077700096FE320068005700900078006380500049
:107780009CFE320068005700900078006480500032
:10779000A1FE32006800570090007800658050001C
:1077A000A7FE320068005700900078006680500005
:1077B000ADFE3200680057009000780067805000EE
:1077C000B3FE3200680057009000780068805000D7
:1077D000B9FE3200680057009000780069805000C0
:1077E000BFFE320068005700900078006A805000A9
:1077F000C5FE320068005700900078006B80500092
:10780000CBFE320068005700900078006C8050007A
:10781000D1FE320068005700900078006D80500063
:10782000D7FE320068005700900078006E8050004C
:10783000DDFE320068005700900078006F80500035
:10784000E3FE32006800570090007800708050001E
:10785000E9FE320068005700900078007180500007
:10786000F8FE3200680057009000780072805000E7
:1078700007FF3200680057009000780073805000C6
:1078800016FF3200680057009000780074805000A6
:107890001BFF320068005700900078007580500090
:1078A0002CFF32006800570090007800768050006E
:1078B00031FF320068005700900078007780500058
:1078C00042FF320068005700900078007880500036
:1078D00048FF32006800570090007800798050001F
:1078E0004EFF320068005700900078007A80500008
:1078F00053FF320068005700900078007B805000F2
:1079000064FF320068005700900078007C805000CF
:1079100075FF32009E3B04000000000040DA2000AA
:10792000801F7800CB0A07002F00B1000080FA000A
:10793000000006000200FA0000002000000F78009E
:1079400060004700900078007C80500009003C00F7
:1079500060004700901F7800ABFD07002F00B100CA
:10796000110020006000470010884000A03C040087
:10797000000000000080FA00000006000200FA008B
:10798000E00047006A00570080087800811F7800F7
:10799000901F780068005700901F7800D0070700FC
:1079A0006F00B1000080FA00000006000000FA003D
:1079B000A2072000E80057001100110007003E0058
:1079C00012062000E80057001100110003003900E2
:1079D000F1FD2F0068005700108860004EB8970036
:1079E0000080FA00000006000200FA0000002000FB
:1079F000000F780068005700900078006000470092
:107A0000108040009040780060C0500013003200A9
:107A1000711080000020200000806000C900DE009E
:107A20000100E00002003200083D040000000000F8
:107A30006800570010007800600147009200400085
:107A4000114078000080FB008010880010002000AA
:107A500012094000FA3C0400000000000080FA0017
:107A6000000006000C00FA0020002000000F780043
:107A70000000200030079800680057009000780050
:107A800066004700108040009040780060C05000C1
:107A90000C003200680057001000780066014700B3
:107AA00012004000904078008180FB006000470099
:107AB0001088680010002000120940003C3D0400BE
:107AC0000000000060004700901F7800F04E2F007B
:107AD000801F780062004700801F7800A7FF070022
:107AE0006F00B1000000200030079800E20047005E
:107AF00066004700108040009040780060C0500051
:107B000011003200E200470066004700500798006D
:107B10001080400040079800104078000080FB0073
:107B2000801F7800A1FF07002F00B100CE00900059
:107B300080487800110020005E009000108840000E
:107B4000763D04000000000062004700801F7800BE
:107B500068005700901F7800404F2F00801F78006A
:107B600040DA2000801F780084FF07008F00B100FA
:107B700040DA2000801F78009BFF07002F00B10033
:107B80000080FA00000006002A00FA0060004700AA
:107B900011502F000E000900315878006F00470087
:107BA00001512F0001000900315878007100470091
:107BB00021512F000100090031587800730047005F
:107BC00041512F001600090031587800600047002D
:107BD000801F7800A3FF07002F00B1004EB8970068
:107BE0000000E000060032006F004700801F7800B0
:107BF0009CFF07002F00B100083E040000000000B9
:107C000071004700801F780096FF07002F00B10029
:107C100073004700801F780092FF07002F00B1001B
:107C20000080FA00000006000000FA00F1EF2F00CB
:107C300060082000108860004EB897000000E00047
:107C40000500320001102000E008200010887000BC
:107C5000323E040000000000F1EF2F00E008200099
:107C600010886000D1FF2F00802120001088600064
:107C70000080FA00000006000000FA00EA00570049
:107C800011007800103B880062804000904078002E
:107C900020032000014878006C0057001000780095
:107CA000003B88000C0007000080FA00000006007E
:107CB0000000FA0040042400801F78006A0057008A
:107CC000B01F7800A01F7800EBFF07006F00B10025
:107CD0000080FA00000006000000FA000500FC0029
:107CE0005C0520003C3B8800AC0A20003C3B88003F
:107CF00061E7A80000000000000000000080FA001A
:107D0000000006000000FA006A005700B01F78006B
:107D1000A01F7800E6FF07004F00B100013B800084
:107D20000000280000806000CF00DE000100E000BD
:107D3000020032008E3E040000000000EA005700FE
:107D400011007800C00088006280400090407800F8
:107D500020032000014878006C00570010007800D4
:107D6000B00088000B0EBB0040002400003B8800E0
:107D7000D9FF0700F1FF2B0000762000108860007B
:107D80000080FA00000006000A00FA006A005700AE
:107D900010007800100798004EB997003200780064
:107DA000A20078002007980031079800000020000A
:107DB000000F780060004700100278006C01570047
:107DC000120052001D003D001E009000901F780020
:107DD0006400470040079800B01F7800A01F78009B
:107DE000C8FF07006F00B1002200200062004700BA
:107DF0001008410022002000CF91DE004E009000CC
:107E00001018410010904900023B8000000028003B
:107E1000000061004F01DE000200E00002003200BD
:107E2000043F040000000000120020006000470032
:107E300010084100DA3E0400000000006C0057000A
:107E4000100078004100DD004EB99700CF80DE00C1
:107E500012194000129148000080FA00000006004C
:107E60000200FA0000002000000F7800CEB8970052
:107E700011007800104178000103200001405100FA
:107E800016003900CEB89700110078001041780034
:107E9000910320000140510010003E0060024700A5
:107EA00094007800A00020000089B900CEB89700A7
:107EB00011007800104078000080FB008000410035
:107EC00000032000008A5000CEB897001000200068
:107ED00091084000363F0400000000001E007800BA
:107EE0000080FA00000006000200FA006800570057
:107EF00010007800000F78001E0078009040780095
:107F000060C050000B0032003EB997001100200005
:107F10006A005700108810000200E00005003200DF
:107F20001100200060004700108840007C3F0400E2
:107F300000000000600047009000780068005700D3
:107F4000108050000080FA00000006000000FA00D7
:107F500002000700FA3F0400000000000400E000F7
:107F600002003A001000070000000600811F7800A0
:107F70000100E00002003D0060001000E0801800F9
:107F80000300E00002003D0060011100E0811900E3
:107F9000050007004F00E00002003B0060001000F9
:107FA000E080180000000600020007000400BE0088
:107FB000000006006022B800060220000000D00089
:107FC0008180D2000482D2008582D2000000A0000D
:107FD0000202520083825A0003003B000202420068
:107FE00083824A000000A1000603E900F3FF3A0083
:107FF000000006000080FA00000006000000FA0001
:10800000020007004C400400000000000400E000F3
:1080100002003A001000070000000600839F68007D
:108020000100E00002003D0060001000E080180048
:108030000300E00002003D0060011100E081190032
:10804000050007004F00E00002003B006000100048
:10805000E0801800000006006022B8000602200040
:108060000000D0008180D2000482D2008582D2003C
:108070000000A0000202520083825A0003003B006D
:108080000202420083824A000000A1000603E900C8
:10809000F3FF3A00000006000080FA00000006002E
:1080A0004C00FA00F077800020279800020420009E
:1080B0007400570010016100020032003079800026
:1080C00020279800740057001000780070016000AD
:1080D00003003200E2FF2F00740057001008610017
:1080E0006E00570010017800620051000600350054
:1080F000440220006E0157001200120002003C00F2
:108100008840040000000000000020001301370038
:108110007400570010007800610160000400320014
:1081200000032000004178009C4004000000000093
:1081300000022000004178006000470002487800FB
:1081400061014700000020000049780074005700DA
:108150001000780062016000290032006C005700B6
:1081600030017800A0017800600051006080590063
:108170000D003D0061014700D00220000049780059
:108180006C01570032007800A200780060191000DE
:1081900060911800120020007000570010081100B4
:1081A0000041040000000000740057001000780037
:1081B000640160000800320061014700B002200045
:1081C00000497800120020007000570010081100CC
:1081D0000041040000000000740057001000780007
:1081E00068016000060032006101470000022000C3
:1081F000004978001200200070005700100811009C
:1082000002022000740057001001610010003200CB
:108210006E005700100178007000510005003A0010
:1082200022002000700057001008110028410400AF
:10823000000000006E005700100178006800510037
:1082400003003A00120020007000570010081100CF
:1082500000002000302798006C00570030017800A3
:10826000A001780060005100608059000A003A00C7
:10827000620047006404200004024700140140002B
:10828000000320000049780010002000140A40007C
:1082900094410400000000006C0057003001780099
:1082A000A001780060005100608059001E0032007B
:1082B000620147006004200000004700502798003A
:1082C00010004100402798001EB997008001EB0084
:1082D0002EB89700BEB897000002EB001BFF070006
:1082E0004204200002014700120140004E2090008D
:1082F00012487800120020005E2090001008410013
:108300001EB997008001EB002EB89700BEB8970009
:108310000002EB0039FF070020BF9F0031BF9F0024
:108320004C410400000000006004200000004700F1
:10833000100278007201570012005200040034004D
:1083400060042000000047001000780070B79F0014
:1083500072005700100178007000570010081100DB
:108360007400570010007800710160000E003A00A0
:108370000EBA97001200200070005700100811007C
:1083800060005200080034004EB99700000220003F
:1083900000497800120020006800570010084100D2
:1083A000B8410400000000001E4090000004E000FE
:1083B00006003200610147004EB89700124878006D
:1083C000120020006800570010084100020220003F
:1083D00074005700100161001D0032006E0057004C
:1083E000100178006800510008003A004EB997006B
:1083F00000032000004978001200200068005700A8
:108400001008410028420400000000006E005700E0
:1084100010017800700051000D003A004EB997002D
:108420000003200000497800E8025700150078009A
:108430006102400044BF9F0012022000E0EF2000D4
:1084400010004100104A780010002000950A4000FA
:108450007400570010007800700160000E003A00B0
:108460000EBA97001200200070005700100811008B
:108470006000520008003400600147004EB89700C9
:1084800012487800120020006800570010084100D0
:1084900030420400000000007EB29700120020006D
:1084A000720057001008110062042000020147000A
:1084B0001200120008003D004EB997000003200092
:1084C00000497800120020006800570010084100A1
:1084D0004C420400000000003E22900012002000E8
:1084E00060042000000047001008110060005200E6
:1084F0000B003400620147006004200000004700C8
:10850000100141004EB89700124878001200200078
:1085100068005700100841006C4204000000000091
:108520000EBA9700120020007000570010081100CA
:1085300060005200080034004EB99700000220008D
:108540000049780012002000680057001008410020
:1085500090420400000000004EB897000080FA002E
:10856000000006001E00FA00F0778000400F98001F
:10857000010420007000570090806000020032006B
:1085800030798000400F980000002000600F9800B4
:1085900000002000500F98007A00470090007800FB
:1085A000668050002E003D007A0047009000780061
:1085B0006080500007003200600047007C014700E7
:1085C00092004000A00320008048780010002000A6
:1085D00012094000E00347007C0347001681430076
:1085E000EA025700150078007A0247009400400024
:1085F000114078000080FB004400DE00F8014700D5
:108600001300400010497800060078001000780040
:1086100061004000600F9800008143000500780071
:10862000900078000400780010804000104078002E
:108630000080FB00EF006000030078001080400025
:108640001049780010002000160B40001100200097
:108650007A00470010884000CC420400000000006F
:108660007000570010007800F00060000F003A0022
:108670002EB99700110020006C00570010881000E0
:10868000FC0047001100110008003D00CEB8970023
:108690000002200080487800110020006800570088
:1086A0001088400038430400000000000000200053
:1086B000500F98007A00470010017800FC00470036
:1086C000110051000D003D00E00047007A00470016
:1086D000908040004EB897001148780011002000AB
:1086E0006800570010884000110020007A00470001
:1086F000108840005A430400000000002EB9970083
:10870000110020006C00570010881000FC0047008A
:108710001100110008003D00CEB8970000022000B3
:108720008048780011002000680057001088400041
:108730007E430400000000004EB897000080FA005D
:10874000000006002800FA0000002000600F9800DA
:1087500000002000400F98007800470010027800C9
:108760006400520082003D0078004700100278004B
:10877000600052000700320060004700FC02470022
:1087800015024000E0022000004A7800100020009E
:10879000950A40006A0057001002780078004700F0
:1087A00010024200144078000080FB00500F980037
:1087B0007A004700100278006000520009003A0079
:1087C00060004700FC02470015024000F07780007F
:1087D000104A780010002000950A4000AE440400C2
:1087E00000000000450620007A02470014801200B5
:1087F0003400350060024700341798007C004700C1
:108800002017980010004200700F980044062000C6
:108810007A00470010179800100078001100090036
:108820000400D800E4EF2000041798001402400070
:108830007E089000144878002E10900010007800F8
:1088400061004000700F9800600F980044062000FF
:108850001E10900010007800110009000400D800DC
:1088600001007800500F9800BE1290007E0A900020
:1088700004824200740F9800A40020001100090037
:108880000400D8000E129000140240007E089000F0
:1088900014487800140020002E10900010084200A8
:1088A0001E10900010027800A200200011000900A4
:1088B0000202D80001007800500F98009C44040088
:1088C000000000007A004700100278006A005200A1
:1088D00019003500600247007C004700101798001F
:1088E00010004200001798007A004700700F9800AF
:1088F00010027800A2002000110009000202D80036
:10890000E4EF2000140240000E109000144878009C
:10891000140020001E109000100842007E089000F5
:1089200010027800A2002000110009000202D80005
:1089300001007800500F9800600047007C0347005A
:1089400096024000F47780007A0047001000420051
:10895000904A780010002000160B40001400200000
:108960007800470010084200AC43040000000000FB
:108970007000570010007800700260000F003A008D
:10898000AEBA9700140020006C00570010081200C7
:108990007C0247001480120008003D004EBA970088
:1089A00000022000004A78001400200068005700F0
:1089B00010084200C0440400000000000000200035
:1089C000400F980078004700900278007C02470032
:1089D000148052000D003D006002470078004700FF
:1089E000100242004EB8970014487800140020008E
:1089F000680057001008420014002000780047006B
:108A000010084200E244040000000000AEBA9700E3
:108A1000140020006C005700100812007C02470070
:108A20001480120008003D004EBA9700000220009A
:108A3000004A780014002000680057001008420027
:108A400006450400000000004EB897000080FA00C0
:108A5000000006000000FA003EB89700CEB897006C
:108A6000100007000081EB00030C07002EB99700EF
:108A700000197800011178002EB89700B001780035
:108A8000200278006A01570032007800A2007800C6
:108A90000301780084017800E40C07000080FA00EC
:108AA000000006000000FA0002000700C6450400AE
:108AB000000000000001BE001F0007000470A700B6
:108AC00003F0A1006509B100160032000D00350069
:108AD0006828E10006003500F0FF2F00F1FF2700B5
:108AE0000300E00013003B00010028000000050027
:108AF00000004000818048008502E900FCFF3A0048
:108B000008003700F88F420002003C008000EB00B4
:108B1000000005008100D1000080D3008502E8003C
:108B2000FCFF3A000300E00002003B006000100080
:108B3000E080180000000600C70ADE00F107B2005E
:108B4000F50FB20008003200E1CF4200020032000F
:108B50000170A00024000500810F700001003200A8
:108B60000408050044000500810F700002003A006F
:108B7000140005008502E9000000400081C04800A3
:108B8000FCFF3B000170A000240005000080FA00FB
:108B9000000006001000FA006C0057001001780079
:108BA0006000510002003D000000200020BF9F0037
:108BB000F40420006C01570012001200020035007E
:108BC000E004200020BF9F0000002000000F78007C
:108BD0000EB99700000020000009780072005700CD
:108BE00010007800500798006A01570032007800A2
:108BF000A20078000200200003002000C90C07003A
:108C00000000E000020035000000200001003700F5
:108C1000100020000000E000080032000EB99700AC
:108C20001000200000097800020020000300280046
:108C30006A00570010186900109069006200470030
:108C400070079800801F78006A005700B01F7800F6
:108C5000A01F78007FFF07006F00B10030BF9F00AA
:108C600041BF9F0004052000720157006C004700BF
:108C7000120842007E009000000178003200780067
:108C8000A20078000200200003002000A50C0700CD
:108C90000000E00002003A00000020000100370060
:108CA000100020000000E000460032000405200013
:108CB000720157006C004700120842006201470031
:108CC00032007800A200780002002000030020009B
:108CD000940C07000000E00002003A0000002000B1
:108CE00001003700100020000000E00022003200E8
:108CF00062004700801F7800020020000312240059
:108D00001E009000AE009000410D0700801F78000B
:108D1000811F78004FFF07006F00B10030079800F7
:108D2000410798006C014700120178006101510071
:108D30007207980062079800F2282C0053CF230096
:108D40007D0C07000200200003122400A50B070081
:108D500054FF0700040320007E01900004494000F6
:108D60007E009000120020006000470010084100C3
:108D70005E4604000000000002052000720057005B
:108D8000100241006C014700120012000B0031007C
:108D90006E0190005E0090001248780012002000E2
:108DA0006A00470010084100120020006C004700D4
:108DB00010084100BC4604000000000036470400D3
:108DC000000000006A01570032007800A20078001D
:108DD00002002000030020000F0C07000000E0004C
:108DE00002003C00000020000100370010002000BD
:108DF0000000E0001D0032003EB89700CEB897009A
:108E00000200200003122400760B070030079800B0
:108E100041079800000178008101780000002000DF
:108E200001F82300FC0B07000000E00002003C00FA
:108E30000000200001003700100020000000E000CA
:108E40000A0032006601470032007800A200780074
:108E500030BF9F0041BF9F0012002000600047000C
:108E600010081100FC4604000000000072005700CA
:108E7000100278006C0157006C0047001208420095
:108E800074005700100178006000510004003A009F
:108E900060004700100178006C0047001008410096
:108EA0001EB99700600047001000780000097800A4
:108EB0006C00470010027800720157001200520047
:108EC000050031007EB197000000200000497800C5
:108ED0007EB09700690037006A00470010027800F2
:108EE0006C0147001200520020003E0002052000E5
:108EF00072005700100241006A0147001200120080
:108F00001A0031003EB89700CEB89700020020004A
:108F100003122400330B070030BF9F0041BF9F00A6
:108F200066014700821F7800801F7800811F78004B
:108F3000C8FE07006F00B10030BF9F0041BF9F0017
:108F40003E009000CE009000D6FE070004032000F3
:108F50005E01900004494000120020006A004700B2
:108F6000100841006C4704000000000002052000CA
:108F700072005700100241006C01470012001200FD
:108F800007003900F2042000720057001001410070
:108F900000002000004978007EB0970037003700BD
:108FA0006C00470010007800500798006E01900098
:108FB00050002000124940006E00900010427800DE
:108FC0009203200002405200280036006E019000FB
:108FD00000032000004978006C0047001002780070
:108FE0007201570012005200090036006C00470061
:108FF00010007800610150006207980002007800BC
:109000001040780061494000324804000000000030
:109010006E01900010032000004978001EB99700EF
:109020001000200012094000740057001001780061
:10903000600051000B003A006A00470010027800FF
:109040007201570012005200030036005E019000CA
:109050000003200000497800120020006A00470049
:1090600010084100DC470400000000005E01900091
:1090700000002000004978007EB097000080FA00D0
:10908000000006005800FA00000020003007980099
:109090006E00570010417800610620000140510029
:1090A0008F003A0000002000801F78006800470011
:1090B000801F780062004700801F78006000470032
:1090C000801F780070005700901F78006A005700DA
:1090D000B01F7800A01F7800AEFE0700EF00B100BF
:1090E000300798001E0090000000E00006003200EB
:1090F000AEB89700D0022000804878001100200010
:109100006C00570010884000BE0090001104E00081
:1091100051003200600047009000780060805000ED
:109120002E003C00AEB89700000320008048780075
:109130006C01570012007800E100400021BF9F0041
:10914000E002200080487800100020001209400052
:109150000000200020079800600047001000780001
:1091600060011000E4004700110011000B003D00F9
:10917000AEB897000003200080487800110020005E
:109180006C00570010884000110020006400470068
:1091900010884000AC48040000000000BE009000B1
:1091A0001104E0000B003200BE0090002EB89700C2
:1091B00011487800110020006C0057001088400012
:1091C000110020006600470010884000CE480400CF
:1091D00000000000284904000000000000002000FA
:1091E00020079800BE0090001104E0001800320033
:1091F0002E019000110020006400470010884000FC
:10920000E00047001100510006003A00AEB8970098
:10921000E002200080487800110020006C00570018
:1092200010884000BE0090002EB8970011487800CA
:10923000110020006C005700108840001100200031
:109240006600470010884000F2480400000000005B
:109250007049040000000000AEB897000003200031
:1092600080487800110020006C00570010884000F2
:1092700070005700900078006080500018003400A3
:10928000AEB89700E002200080487800110020006E
:109290006C00570010884000000020002007980054
:1092A0006400470010017800F000570011005100E1
:1092B0000B003D00AEB89700000320008048780006
:1092C000110020006C0057001088400011002000A1
:1092D000640047001088400050490400000000006E
:1092E000AEB8970000002000804878000080FA00A7
:1092F000000006000200FA00CEB897001104E0005A
:10930000190032004EB8970010417800E1022000A9
:109310000140510001003A003A0037004EB8970072
:109320001041780051062000014051000700320032
:109330004EB89700104178005104200001405100C0
:1093400002003200AA49040000000000B4490400F1
:109350000000000011002000680057001088400045
:109360007C49040000000000CEB897001104E00022
:109370001B00320068005700901F780005040700AA
:109380002F00B100000F78006000470090007800C7
:10939000608050000D003400E001470013007800A9
:1093A000E100400068005700108140009000780004
:1093B0000300780010804000104978001000200061
:1093C00093091000C449040000000000CEB89700C3
:1093D000E002200080487800024A040000000000FB
:1093E000CEB89700E002200080487800680057005F
:1093F00010007800E100400041BF9F000000200005
:10940000804878000080FA00000006000200FA00A0
:10941000CEB897001104E0000A0032004EB8970061
:1094200010417800E10220000140510005003200A7
:10943000110020006800570010884000084A04000E
:10944000000000004EB9970011002000680057008E
:10945000108840001204E00037003200CEB89700B8
:109460001104E0000F0032004EB897001041780060
:1094700051062000014051000A0032004EB897000A
:1094800010417800510420000140510005003200D5
:109490001100200068005700108840002E4A040088
:1094A00000000000E800570011007800000F78006D
:1094B00010002000910810004EB89700104178006D
:1094C000010320000140510005003A001100200076
:1094D00068005700108810005C4A0400000000007B
:1094E0004EB8970010417800E10220000140510081
:1094F00003003A0011002000680057001088100097
:109500006800570010007800E101400043BF9F0051
:109510001E01780011002000600047001088400004
:1095200092497800CEB897001104E00002003200A2
:10953000804A0400000000000080FA0000000600DD
:109540005600FA00740057001000780070016000A7
:1095500003003200E2FF2F00740057001008610082
:1095600074005700100078006101600004003200B0
:109570000003200000417800C44A040000000000FD
:109580000002200000417800000520000000470094
:109590000248780012052000020147000000200068
:1095A00000497800740057001000780062016000E4
:1095B000330032006C01570032007800A2007800BE
:1095C0000200200003002000560A07000000E0000F
:1095D00002003500000020000100370010002000CC
:1095E0000000E0000E0032001205200002014700DA
:1095F000D00220000049780002002000030028006B
:109600006C005700101869001090690012002000CB
:109610006E00570010081100404B040000000000CD
:1096200074005700100078006401600009003200E7
:109630001205200002014700B00220000049780016
:10964000120020006E00570010081100404B04006B
:1096500000000000740057001000780068016000EE
:10966000070032001205200002014700000220001E
:1096700000497800120020006E0057001008110009
:1096800070005700100178006000510004003D0098
:109690006000200000BF9F00664B04000000000037
:1096A00070005700100178006000510007003A0078
:1096B00072005700104278007206200002405200EB
:1096C00002003A001000200000BF9F007000570009
:1096D000901F780072005700104078000080FB0057
:1096E000801F780060004700801F78006C005700E2
:1096F000B01F7800A01F780062FE0700AF00B10025
:1097000002022000740057001001610008003200BE
:1097100070005700100178006000510004003A000A
:1097200060004700801F7800F2FE07002F00B100A4
:10973000720057001042780072062000024052006A
:1097400008003A0002022000740057001001610076
:1097500004003A0060004700801F78002BFF0700DC
:109760002F00B10060004700801F78000903070048
:109770002F00B100102F98006E0157001209100041
:109780007400570010007800710160000E003A006C
:109790001EBA9700120020006E005700100811003A
:1097A00060005200080034004EB99700000220000B
:1097B000004978001200200068005700100841009E
:1097C000C84B0400000000001ED090000004E00020
:1097D0000700320012052000020147004EB8970032
:1097E000124878001200200068005700100841005D
:1097F0007400570010007800700160000F003A00FC
:109800001EBA9700120020006E00570010081100C9
:1098100060005200090034000205200002014700E8
:109820004EB89700124878001200200068005700D8
:1098300010084100004C040000000000000020005F
:10984000202F9800400520000000470010027800FB
:109850002205200002014700120052000F003D00C7
:109860006001470040052000000047001001410052
:109870004EB8970012487800120020006800570088
:1098800010084100120020004005200000004700A1
:1098900010084100224C0400000000001EBA97008E
:1098A000120020006E0057001008110060005200E6
:1098B000080034004EB997000002200000497800EB
:1098C0001200200068005700100841004E4C0400B0
:1098D000000000004EB897000080FA00000006006B
:1098E0001E00FA0060004700B1522F000600090078
:1098F000315878006800570010007800100F980069
:109900003EB997001204E000990232003EB8970079
:10991000904178005202200002C05100080032003D
:109920003EB997001E0890001248780012002000EF
:109930007200470010084100AE5104000000000012
:1099400000002000300F9800120020006A0057002D
:1099500010084100E04C040000000000020120005B
:109960007600470010087100A44C040000000000BD
:10997000420020007600470010087100A44C04004B
:1099800000000000820020007600470010087100EF
:10999000A44C0400000000000202200076004700F2
:1099A00010087100A44C0400000000001200200008
:1099B0007600470010087100A44C0400000000006D
:1099C0003EB8970090417800D202200002C05100BA
:1099D000E2FF32003EB8970090417800B2022000CA
:1099E00002C05100E2FF32003EB89700904178007B
:1099F0000202200002C05100E2FF32003EB8970090
:109A0000904178003202200002C05100E2FF320093
:109A10003EB89700904178000203200002C0510038
:109A2000E2FF3200F0FF2F00400F98003EB8970091
:109A3000904178000203200002C051000C00390060
:109A40003EB89700904178009203200002C0510078
:109A500007003E006A005700801F780000F90700E9
:109A60002F00B100400F9800664D04000000000078
:109A70003EB8970090417800A202200002C0510039
:109A800012003A00120020006A005700100841003E
:109A9000AEB997002EB997002000200012091000DF
:109AA0001300780010017800420F98006000510008
:109AB00006003D00780147001200780060091000A0
:109AC000020120007600470010087100F0FF2F000F
:109AD000500F98003EB8970090417800E2022000B5
:109AE00002C0510029003A006A00570010007800B7
:109AF0006100400030BF9F009041780002032000C9
:109B000002C051000C0039003EB897009041780027
:109B10009203200002C0510007003E006A00570077
:109B2000801F7800CEF807002F00B100500F98007A
:109B3000BA4D0400000000003EB897009041780044
:109B4000A202200002C051000A003A0012002000C8
:109B50006A00570010084100AEB997002EB997006F
:109B60002000200012091000130178001200780074
:109B7000500F98007A0047001001780060005100F3
:109B800002003D0000002000500F9800F0FF2F0061
:109B9000600F98003EB89700904178008206200040
:109BA00002C051000C0032003EB89700904178008E
:109BB000C206200002C05100070032003EB89700E4
:109BC00090417800C204200002C05100020032001F
:109BD000FA4D0400000000003EB9970012407800E2
:109BE0000080FB00600F9800120020006A00570000
:109BF00010084100A0002000000F980052500400FF
:109C0000000000007600470010007800700160003E
:109C10000E003A0078004700100078006101500003
:109C2000420F980060005100080034001E099000A7
:109C30000002200000497800120020007200470056
:109C4000100841000A4E040000000000AEB9970061
:109C50002EB997002000200012091000130178008F
:109C60001E08900012487800120020007200470081
:109C70001008410078004700100078006101500092
:109C8000420F980060005100080034001E09900047
:109C900000022000004978001200200072004700F6
:109CA000100841003A4E040000000000AE510400CC
:109CB00000000000AEB997002EB9970020002000E8
:109CC000120910001300780010017800220F98008C
:109CD0006000510002003A0060004700200F980029
:109CE0007A004700901F780074004700901F7800AA
:109CF0007DF807004F00B10040079800760047004C
:109D000010007800700160000F003A00CE0990004A
:109D10001200200078004700100811006801470079
:109D20001280110008003D001E0990000002200072
:109D3000004978001200200072004700100841001E
:109D4000864E04000000000000002000700798000C
:109D50006E004700900178006801470012805100B2
:109D60000E003D002E0990001E0890001248780059
:109D7000120020007200470010084100120020006D
:109D80007400470010084100120020006E004700D8
:109D900010084100A84E040000000000CE09900009
:109DA00012002000780047001008110068014700E9
:109DB0001280110008003D001E09900000022000E2
:109DC000004978001200200072004700100841008E
:109DD000CE4E040000000000AE5104000000000060
:109DE000F3FF2F00780147001280110005003A00B0
:109DF00040002000400F980012002000760047002D
:109E00001008710076004700901F78007A00470024
:109E1000901F780078004700901F78000001200014
:109E2000801F7800AEB997002EB99700200020005F
:109E30001209100013007800100078008000EB0079
:109E4000801F7800811F780072004700901F780003
:109E500093F80700EF00B100100F9800AE51040016
:109E600000000000C30620007C01470012801100A2
:109E70000F003A00AEB997002EB9970020002000DD
:109E8000120910001300780090017800720047005A
:109E90001001780068005700100051008000EB00AE
:109EA00080197800811178006C4F040000000000D8
:109EB000AEB997002EB997002000200012091000BB
:109EC00013007800900178007200470010017800BC
:109ED0006800570090095100AE51040000000000D6
:109EE000020420007600470010087100C30620001D
:109EF0007C0147001280110013003A0076004700F1
:109F0000901F78007A004700901F78007800470083
:109F1000901F7800AEB997002EB99700200020005E
:109F20001209100013007800901F7800720047009B
:109F3000901F78008BF90700AF00B100100F980058
:109F4000C64F04000000000076004700901F780014
:109F50007A004700901F780078004700901F780033
:109F6000AEB997002EB9970020002000120910000A
:109F700013007800901F780072004700901F78004F
:109F8000F0F90700AF00B100100F9800AE510400C7
:109F90000000000080002000000F98000051040025
:109FA0000000000002042000760047001008710045
:109FB00000012000000F9800005104000000000084
:109FC00022002000760047001008710000510400B4
:109FD000000000007600470010007800620070006A
:109FE000801F78003EB9970012407800801F7800EB
:109FF0007A004700901F780078004700901F780093
:10A00000AEB997002EB99700400020001209100049
:10A0100013007800B01F7800A01F7800720047007E
:10A02000901F780046FD0700EF00B100100F980068
:10A03000AE510400000000003EB897009041780047
:10A040005202200002C05100060032001E0990009A
:10A0500050022000004978001200200072004700E2
:10A06000100841003EB997001204E00008003200D9
:10A070003EB997001E089000124878001200200098
:10A0800072004700100841004E500400000000001C
:10A09000120020006A00570010081100AE510400A1
:10A0A000000000003EB89700904178003206200082
:10A0B00002C05100D3FE32003EB8970090417800B4
:10A0C0003207200002C05100FAFE32003EB897006D
:10A0D000904178000207200002C0510040FF32008A
:10A0E0003EB8970090417800E206200002C051007F
:10A0F0005CFF32003EB897009041780012042000C7
:10A1000002C0510076FF32003EB8970090417800BF
:10A110001206200002C0510074FF32003EB89700C2
:10A1200090417800F206200002C0510099FF3200F1
:10A130003EB89700904178008205200002C051008F
:10A1400098FF32003EB897009041780082072000C7
:10A1500002C0510096FF32003EB89700904178004F
:10A160004206200002C0510095FF32003EB8970021
:10A17000904178009206200002C0510090FF32000A
:10A180003EB89700904178005207200002C051006D
:10A190008EFF32003EB897009041780052042000B4
:10A1A00002C051008BFF32003EB89700904178000A
:10A1B0007204200002C0510086FF32003EB89700B2
:10A1C000904178005206200002C0510081FF320009
:10A1D0003EB89700904178006206200002C051000E
:10A1E0007CFF32003EB89700904178007206200054
:10A1F00002C0510077FF32001C5004000000000034
:10A20000C30620007C014700128011000B003A00B9
:10A21000AEB997002EB99700400020001209100037
:10A220001301780032007800A200780050079800EF
:10A23000610798008E510400000000008306200092
:10A240007C014700128011001C003A007600470094
:10A2500010007800620160000C003200AEB9970077
:10A260002EB9970010002000120910001301780089
:10A27000124078000000FB00CF80DE0050079800FD
:10A28000610798005A51040000000000AEB9970021
:10A290002EB9970010002000120910001301780059
:10A2A000124078000080FB008000EB00500798000F
:10A2B000610798008E5104000000000076004700FE
:10A2C00010007800620160000B003200AEB9970008
:10A2D0002EB9970020002000120910001301780009
:10A2E00012007800CF80DE005007980061079800C8
:10A2F0008E51040000000000AEB997002EB99700FF
:10A3000020002000120910001301780012007800CC
:10A310008000EB0050079800610798007600470026
:10A32000901F78007A004700901F7800780047005F
:10A33000901F780070004700901F78006A00470067
:10A34000B01F7800A01F780072004700901F7800AF
:10A3500053F70700EF00B100100F98001200200023
:10A360006A00570010084100804C04000000000003
:10A370001E0990000000200000497800720047008C
:10A380001001780068005700100051000080FA00AA
:10A39000000006000200FA00680057001000780074
:10A3A000000F78001E0178001100200060004700B7
:10A3B000108840001204E00002003200D251040074
:10A3C000000000006000470090007800680057001F
:10A3D00010805000610050000080FA00000006006C
:10A3E000C822A90020C2A9002022AF00F451040015
:10A3F00000000000F00F2000201188002002AE00B5
:10A40000FE5104000000000020118000F10F200028
:10A410000104E100F3FF3A0020C2A9002022AF00AE
:10A420000E520400000000000000EB002011880024
:10A430002002AE001852040000000000201180002D
:10A44000F000B200110020000008DD00C822A800C2
:10A45000000006000200FA0068005700901F780014
:10A46000CCFF07002F00B100000F7800DCFF0700D1
:10A4700060014700920010000200360036520400CE
:10A4800000000000C822A900680057009000780072
:10A49000314078000080FB00060032002022AF002F
:10A4A0004E520400000000002011880048520400B1
:10A4B00000000000C822A8000080FA00000006008A
:10A4C0003E00FA00E000470068005700800878006E
:10A4D000811F7800901F780062004700801F78007D
:10A4E000FFFC07006F00B10062004700801F78008A
:10A4F000D8FF07002F00B1000080FA00000006001E
:10A500000000FA0068005700901F780020532F00C9
:10A51000801F7800EAFF07004F00B1000080FA00BA
:10A520000000060050042000801F7800F4FF0700A0
:10A530002F00B100000006000A00FA00307380000E
:10A5400010079800820C20008001EB00A0E620009C
:10A5500030021100A0821900E2D020003200120067
:10A5600022801A000F003D0032738000E0C32000FB
:10A5700010014100327388006000510002003D006C
:10A580000000200030738800327380007C0051008E
:10A5900002003400C001200030738800045D040014
:10A5A00000000000820C20008001EB00A0E62000EB
:10A5B00030024100A0824900E2D0200032001200A7
:10A5C00022801A000F00340032738000E0C32000A4
:10A5D00010015100327388006000510002003D00FC
:10A5E0000000200030738800327380007C0051002E
:10A5F00002003400C001200030738800045D0400B4
:10A600000000000000002000000F7800820C2000F5
:10A610008001EB00E0E6200030024100A08249000A
:10A6200062D020003200120022801A0004003400A0
:10A6300010002000000F78003653040000000000D6
:10A64000820C20008001EB00E0E6200030021100C7
:10A65000A082190062D020003200120022801A006D
:10A6600002003D00F0FF2F00000F7800600047005F
:10A670001001780000C420001091B900020F78008A
:10A6800060005100E0043200327380007C00510011
:10A69000060032001000200040738800C001200036
:10A6A000801F780058F207002F00B1004C5C0400B6
:10A6B00000000000026080001360800000002000A5
:10A6C00001F82300170607000000E0000200340034
:10A6D0000000200001003700100020000000E00012
:10A6E0000600320060004700100178006000510051
:10A6F00002003D00A653040000000000026080003C
:10A700001360800000F82400317C2400C20507009B
:10A710000000E00002003C000000200001003700C3
:10A72000100020000000E00006003200600047003A
:10A73000100178006000510002003400A6530400AC
:10A7400000000000B8530400000000001E00780064
:10A75000CF80DE000081EB00C704070002608000AC
:10A7600013608000F4050700006088001160880015
:10A77000FE5C040000000000226080003360800066
:10A78000A0702D0031C22300E60507000000E000A4
:10A7900002003400000020000100370010002000FB
:10A7A0000000E00006003200600047001001780061
:10A7B0006000510002003D00085404000000000049
:10A7C00022608000336080000000200001F8230038
:10A7D000910507000000E00002003C00000020009E
:10A7E00001003700100020000000E00006003200E9
:10A7F0006000470010017800600051000200340042
:10A800000854040000000000205404000000000070
:10A810001E007800CF80DE000081EB009604070068
:10A82000A2702D0033C22300EE04070022608000D6
:10A8300033608000C0050700206088003160880018
:10A84000FE5C040000000000426080005360800055
:10A85000D0CC2C00C1E42300B20507000000E000CA
:10A86000020034000000200001003700100020002A
:10A870000000E00006003200600047001001780090
:10A880006000510002003D00705404000000000010
:10A89000426080005360800030332300F1192400AF
:10A8A0005D0507000000E00002003C000000200001
:10A8B00001003700100020000000E0000600320018
:10A8C0006000470010017800600051000200340071
:10A8D00070540400000000008854040000000000D0
:10A8E0001E007800CF80DE000081EB0062040700CC
:10A8F000D2CC2C00C3DC2300BA04070042608000E5
:10A90000536080008C05070040608800516088001B
:10A91000FE5C0400000000006260800061005100E5
:10A92000060034006000470010017800600051000C
:10A9300002003D00B654040000000000540920004D
:10A94000C2C020001200120006003D006000470057
:10A95000100178006000510002003400B654040079
:10A9600000000000BE54040000000000600047002A
:10A9700010017800C0C0200010084100FE5C0400F7
:10A9800000000000726080008360800000002000F2
:10A9900001F82300630507000000E0000200350015
:10A9A0000000200001003700100020000000E0003F
:10A9B000060032006000470010017800600051007E
:10A9C00002003D000E55040000000000726080008F
:10A9D0008360800000F82400317C24000E0507000D
:10A9E0000000E00002003C000000200001003700F1
:10A9F000100020000000E000060032006000470068
:10AA00001001780060005100020034000E5504006F
:10AA10000000000020550400000000001E00780027
:10AA2000CF80DE000081EB0013040700726080001D
:10AA300083608000400507007060880081608800A6
:10AA4000FE5C04000000000092608000A3608000B3
:10AA5000D0CC2C00C1DC2300320507000000E00050
:10AA60000200350000002000010037001000200027
:10AA70000000E0000600320060004700100178008E
:10AA80006000510002003D0070550400000000000D
:10AA900092608000A3608000D0CC2C00712C240038
:10AAA000DD0407000000E00002003C000000200080
:10AAB00001003700100020000000E0000600320016
:10AAC000600047001001780060005100020034006F
:10AAD00070550400000000008855040000000000CC
:10AAE0001E007800CF80DE000081EB00E20307004B
:10AAF000D2CC2C00C3DC23003A0407009260800013
:10AB0000A36080000C05070090608800A1608800A9
:10AB1000FE5C040000000000B0608000C1608000A6
:10AB20000200200003002000BB0407000000E0003A
:10AB300002003C000000200001003700100020004F
:10AB40000000E000060032006000470010017800BD
:10AB50006000510002003D00D855040000000000D4
:10AB6000B2608000C3608000000020004124240007
:10AB7000A90407000000E00002003C0000002000E3
:10AB800001003700100020000000E0000600320045
:10AB9000600047001001780060005100020034009E
:10ABA000D855040000000000EA5504000000000031
:10ABB0001E007800CF80DE000081EB00AE030700AE
:10ABC000B2608000C3608000DB040700B0608800D2
:10ABD000C1608800FE5C040000000000D2608000BC
:10ABE000E3608000D0CC2C00C1DC2300CD04070042
:10ABF0000000E000020035000000200001003700E6
:10AC0000100020000000E000060032006000470055
:10AC1000100178006000510002003D003A56040027
:10AC200000000000D2608000E3608000D0CC2C00E7
:10AC3000712C2400780407000000E00002003C00B2
:10AC40000000200001003700100020000000E0009C
:10AC500006003200600047001001780060005100DB
:10AC6000020034003A56040000000000525604006E
:10AC7000000000001E007800CF80DE000081EB00A5
:10AC80007D030700D2CC2C00C3DC2300D5030700D2
:10AC9000D2608000E3608000A7040700D0608800D5
:10ACA000E1608800FE5C040000000000F2608000AB
:10ACB00003618000D0CC2C00C1DC23009904070084
:10ACC0000000E00002003500000020000100370015
:10ACD000100020000000E000060032006000470085
:10ACE000100178006000510002003D00A2560400EF
:10ACF00000000000F260800003618000D0CC2C00D6
:10AD0000712C2400440407000000E00002003C0015
:10AD10000000200001003700100020000000E000CB
:10AD2000060032006000470010017800600051000A
:10AD300002003400A256040000000000BA560400CD
:10AD4000000000001E007800CF80DE000081EB00D4
:10AD500049030700D2CC2C00C3DC2300A103070069
:10AD6000F26080000361800073040700F0608800D7
:10AD700001618800FE5C040000000000106180009A
:10AD8000216180000200200003002000220407004F
:10AD90000000E00002003C0000002000010037003D
:10ADA000100020000000E0000600320060004700B4
:10ADB000100178006000510002003D000A570400B5
:10ADC000000000001261800023618000000020006C
:10ADD00041242400100407000000E00002003C00B1
:10ADE0000000200001003700100020000000E000FB
:10ADF000060032006000470010017800600051003A
:10AE0000020034000A570400000000001C57040030
:10AE1000000000001E007800CF80DE000081EB0003
:10AE200015030700126180002361800042040700BF
:10AE30001061880021618800FE5C040000000000B1
:10AE400032618000436180000000200001F823008F
:10AE5000340407000000E00002003500000020007C
:10AE600001003700100020000000E0000600320062
:10AE700060004700100178006000510002003D00B2
:10AE80006C570400000000003261800043618000C4
:10AE900000002000612C2400DF0307000000E00018
:10AEA00002003C00000020000100370010002000DC
:10AEB0000000E0000600320060004700100178004A
:10AEC00060005100020034006C57040000000000D4
:10AED0007E570400000000001E007800CF80DE00D6
:10AEE0000081EB00E40207003261800043618000D2
:10AEF000110407003061880041618800FE5C040095
:10AF0000000000005261800063618000D0CC2C0002
:10AF1000C1DC2300030407000000E000020035004C
:10AF20000000200001003700100020000000E000B9
:10AF300006003200600047001001780060005100F8
:10AF400002003D00CE570400000000005261800066
:10AF500063618000D0CC2C00712C2400AE0307006C
:10AF60000000E00002003C0000002000010037006B
:10AF7000100020000000E0000600320060004700E2
:10AF8000100178006000510002003400CE57040028
:10AF900000000000E6570400000000001E007800DA
:10AFA000CF80DE000081EB00B3020700D2CC2C0082
:10AFB000C3DC23000B030700526180006361800043
:10AFC000DD0307005061880061618800FE5C0400B9
:10AFD000000000007261800083618000000020009A
:10AFE00001F82300CF0307000000E0000200350055
:10AFF0000000200001003700100020000000E000E9
:10B000000600320060004700100178006000510027
:10B0100002003D003658040000000000726180000C
:10B020008361800000002C00914724007A03070010
:10B030000000E00002003C0000002000010037009A
:10B04000100020000000E000060032006000470011
:10B0500010017800600051000200340036580400EE
:10B060000000000048580400000000001E007800A6
:10B07000CF80DE000081EB007F020700726180005C
:10B0800083618000AC0307007061880081618800E3
:10B09000FE5C040000000000B2618000C36180001B
:10B0A0000000200001F823009E0307000000E000DC
:10B0B00002003500000020000100370010002000D1
:10B0C0000000E00006003200600047001001780038
:10B0D0006000510002003D0098580400000000008C
:10B0E000B2618000C361800000002000612C240058
:10B0F000490307000000E00002003C0000002000BF
:10B1000001003700100020000000E00006003200BF
:10B110006000470010017800600051000200340018
:10B120009858040000000000AA5804000000000025
:10B130001E007800CF80DE000081EB004E02070089
:10B14000B2618000C36180007B030700B0618800AA
:10B15000C1618800FE5C0400000000009261800074
:10B16000A36180000000200001F823006D030700A8
:10B170000000E00002003500000020000100370060
:10B18000100020000000E0000600320060004700D0
:10B19000100178006000510002003D00FA580400E0
:10B1A0000000000092618000A36180000000200088
:10B1B00031332400180307000000E00002003C00C7
:10B1C0000000200001003700100020000000E00017
:10B1D0000600320060004700100178006000510056
:10B1E00002003400FA580400000000000C5904006A
:10B1F000000000001E007800CF80DE000081EB0020
:10B200001D02070092618000A36180004A030700CD
:10B2100090618800A1618800FE5C040000000000CD
:10B22000D2618000E3618000000020000112240050
:10B230003C0307000000E000020035000000200091
:10B2400001003700100020000000E000060032007E
:10B2500060004700100178006000510002003D00CE
:10B260005C59040000000000D2618000E3618000AE
:10B2700000C02300C1612400E70207000000E000D5
:10B2800002003C00000020000100370010002000F8
:10B290000000E00006003200600047001001780066
:10B2A00060005100020034005C59040000000000FE
:10B2B0007259040000000000A20020006000470056
:10B2C0001090B900CF80DE000081EB00EA0107009A
:10B2D000D2618000E361800017030700D06188001D
:10B2E000E1618800FE5C040000000000F261800063
:10B2F0006000510006003400600047001001780033
:10B300006000510002003D009E5904000000000052
:10B31000F26180006000510006003D0060004700BF
:10B320001001780060005100020034009E590400B2
:10B3300000000000A4590400000000006000470065
:10B3400010007800F0618800FE5C0400000000003E
:10B350000262800060005100060034006000470077
:10B36000100178006000510002003D00D059040037
:10B3700000000000026280006000510006003D00F5
:10B3800060004700100178006000510002003400A6
:10B39000D059040000000000D6590400000000004D
:10B3A000600047001000780000628800FE5C040026
:10B3B00000000000126280006000510006003400AE
:10B3C00060004700100178006000510002003D005D
:10B3D000025A040000000000126280006000510068
:10B3E00006003C006000470010017800600051003A
:10B3F00002003400025A0400000000000A5A04004F
:10B4000000000000600047001001780020C4200008
:10B4100010084100FE5C0400000000002262800071
:10B420006000510006003400600047001001780001
:10B430006000510002003D00385A04000000000086
:10B4400024628000823E20000200520006003D007F
:10B4500060004700100178006000510002003400D5
:10B46000385A040000000000405A040000000000A8
:10B47000600047001001780040C42000100841001F
:10B48000FE5C040000000000326280006000510099
:10B490000600340060004700100178006000510091
:10B4A00002003D006C5A040000000000326280007F
:10B4B0006000510006003C00600047001001780069
:10B4C00060005100020034006C5A040000000000CB
:10B4D000785A040000000000600047001001780066
:10B4E00060C420001008410098EE070011F1070029
:10B4F000FE5C040000000000426280006000510019
:10B500000600340060004700100178006000510020
:10B5100002003D00A65A04000000000044628000C2
:10B52000C21220000200520006003D0060004700E9
:10B53000100178006000510002003400A65A040097
:10B5400000000000AE5A0400000000006000470048
:10B550001001780080C4200010084100FE5C040047
:10B5600000000000600047001001780060005100FA
:10B570000600340000002000307088001000200019
:10B58000801F780080F107002F00B100FE5C0400EE
:10B59000000000005262800063628000C05A2C00EC
:10B5A000717223005F0207000000E0000200350016
:10B5B0000000200001003700100020000000E00023
:10B5C0000600320060004700100178006000510062
:10B5D00002003D00165B0400000000005262800083
:10B5E000636280000000200001F823000A020700C7
:10B5F0000000E00002003C000000200001003700D5
:10B60000100020000000E00006003200600047004B
:10B61000100178006000510002003400165B040045
:10B62000000000002E5B0400000000001E007800F7
:10B63000CF80DE000081EB000F010700C25A2C0012
:10B64000737223006701070052628000636280000A
:10B65000390207005062880061628800FE5C0400C5
:10B66000000000007262800083628000F0262100EA
:10B6700031A823002B0207000000E0000200350083
:10B680000000200001003700100020000000E00052
:10B690000600320060004700100178006000510091
:10B6A00002003D007E5B040000000000726280002A
:10B6B000836280000000200001F82300D60107000B
:10B6C0000000E00002003C00000020000100370004
:10B6D000100020000000E00006003200600047007B
:10B6E0001001780060005100020034007E5B04000D
:10B6F00000000000965B0400000000001E007800BF
:10B70000CF80DE000081EB00DB000700F226210085
:10B7100033A8230033010700726280008362800037
:10B72000050207007062880081628800FE5C0400E8
:10B7300000000000926280006000510006003400AA
:10B7400060004700100178006000510002003D00D9
:10B75000C45B0400000000008402200022C5200019
:10B760001200120006003D00600047001001780042
:10B770006000510002003400C45B040000000000BF
:10B78000CE5B040000000000926280006000470071
:10B790001000410090628800C0708800FE5C0400C8
:10B7A00000000000600047001000780061005000B9
:10B7B00002003200000020000100370010002000CD
:10B7C000B0628800FE5C04000000000060004700DA
:10B7D00010007800610050000200320000002000DC
:10B7E0000100370010002000A0628800801F780050
:10B7F0000DF107002F00B100FE5C04000000000006
:10B800006000470010017800600051001E00340005
:10B8100000C02F00F1072000300798004107980072
:10B820000000200020079800640047001001780005
:10B830007B00510011003D006400470010007800BB
:10B840004201DD0080F22000020140006200410060
:10B85000901F7800921F780066004700801F7800D4
:10B8600049F107006F00B10012002000640047009A
:10B8700010084100145C04000000000000002000DB
:10B88000407388002BF00700FE5C040000000000FD
:10B89000FE5C040000000000327380006000510074
:10B8A00084FB32003273800061005100B2FB320031
:10B8B0003273800062005100E3FB3200327380007B
:10B8C0006300510014FC32003273800064005100A8
:10B8D0002CFC320032738000650051005AFC3200AB
:10B8E00032738000660051008BFC3200327380009E
:10B8F00067005100B9FC32003273800068005100CB
:10B90000EAFC320032738000690051001BFD3200F6
:10B91000327380006A00510049FD320032738000AA
:10B920006B00510077FD3200327380006C005100D3
:10B93000A8FD3200327380006D005100D6FD320048
:10B94000327380006E00510004FE320032738000BA
:10B950006F00510032FE32003273800070005100DF
:10B9600062FE3200327380007100510078FE3200B6
:10B9700032738000720051008EFE320032738000FC
:10B9800073005100A5FE3200327380007400510034
:10B99000BDFE32003273800075005100D6FE3200C9
:10B9A0003273800076005100EEFE32003273800068
:10B9B00077005100F7FE32003273800078005100AA
:10B9C00028FF3200327380007900510059FF3200A5
:10B9D000327380007A00510072FF320032738000AF
:10B9E0007B00510079FF3200327380007C005100EF
:10B9F00083FF3200485C040000000000660EF8007F
:10BA000081ED07002F00B1006200470010027800AE
:10BA100062E6200012005200070032006200470078
:10BA2000901F780078ED07002F00B100660EF80037
:10BA300075ED07002F00B100BAFA07000080FA0088
:10BA4000000006000000FA004EB89700BEB897004C
:10BA50000000E00004003200FA3F0900000000008E
:10BA60000000E900FAFF3700018009000000000033
:10BA70000080FA00000006000000FA000200070043
:10BA8000EE5D0400000000000200E00006003A0045
:10BA90000005EB000100E0000F003E000000E000A8
:10BAA000270032000C003700010578000100E0009B
:10BAB0000400350008003C000000E00020003200D7
:10BAC0000500370060001000E080180002003B0015
:10BAD00001F02C001A0037000004BE006011B8000D
:10BAE0006B0920000982CF00020039000882CF00D4
:10BAF0000441B000694252000E00320008003B00D1
:10BB000082817100610164008904D1000884D3003E
:10BB10008B05E8000442E800F9FF3A000500370011
:10BB20000804440089844C008B05E9000442E900C4
:10BB3000FBFF3A00030007000AF0A70001F0A00095
:10BB40000000060081002000618055000B003D00D0
:10BB50000B00200061FE2F000100E1001D003400F9
:10BB600082817100610164008904D1000884D300DE
:10BB70000000E800FAFF3A00710020006100640054
:10BB800003007000020060000900320061044400FC
:10BB9000E0844C000988A500050032008B05E80010
:10BBA0006808E10002003A008904D1000884D3004B
:10BBB000F20F20000258E10005003D00C75DDD00E6
:10BBC000F907B200898075000800780000000600BF
:10BBD0000BF827008B007800000005000080FA00B9
:10BBE000000006000000FA0002000700085F0400E1
:10BBF00000000000889FBE008A9FBE008C1F780056
:10BC0000300007003700330003866C006450E10009
:10BC1000240032006420E100270032006150E1007E
:10BC2000220032006120E100210032008B854200B9
:10BC3000EB07B1000134B800003AB8000804420034
:10BC400089844A00013AB8000030B800888040007A
:10BC500009014A00040033000000400081804800D0
:10BC6000020149008B05E900C909DD00830170006C
:10BC70000100320013002000C814DE004814DD006B
:10BC80004709DE001200B200C808DE000884700018
:10BC90002400070001F0A1000CF0A70001F0A000B3
:10BCA000190037006120E1001B0032000801BE00CE
:10BCB0000200BE00F7FF37006150E100FCFF3A00D0
:10BCC000150037000004BE003C0007000003BE0062
:10BCD0000405BE000200BE0038000700844F750056
:10BCE000000006000200BE006450E10005003600BE
:10BCF0006420E100020036000968A30001003A0058
:10BD00000800BE000160A0004F0678004F05BE008D
:10BD10004F04BE0000000600F0FF2F00F1FF2700D7
:10BD2000F9FF370081002000618055000B003D00C5
:10BD30000B00200061FE2F000100E1001D00340017
:10BD400082817100610164008904D1000884D300FC
:10BD50000000E800FAFF3A00710020006100640072
:10BD6000030070000200600009003200610444001A
:10BD7000E0844C000988A500050032008B05E8002E
:10BD80006808E10002003A008904D1000884D30069
:10BD9000F20F20000258E10005003D00C75DDD0004
:10BDA000F907B200898075000800780000000600DD
:10BDB0000BF827008B00780000000500C70ADE00A2
:10BDC000F107B200F50FB20008003200E1CF4200E7
:10BDD000020032000170A00024000500810F7000F5
:10BDE000010032000408050044000500810F7000C6
:10BDF00002003A00140005008502E900000040003E
:10BE000081C04800FCFF3B000170A0002400050039
:10BE10000080FA00000006000000FA00F4FF2F0086
:10BE2000070007000080FA00000006000000FA008A
:10BE300003F0A200400007000080FA0000000600A6
:10BE40000000FA00020007008E5F040000000000FE
:10BE5000841F7800140007004F00780011003300A1
:10BE6000F0FF2F00838F6C0006003B000405650087
:10BE70000A00A7000800370009F0A6001000200003
:10BE800008003700820F5400838F5C0003003900E4
:10BE90001000200001003E000000200009F0A70073
:10BEA0000000EA00000006000004BE0006000700D3
:10BEB0000003BE000405BE000200BE000200070031
:10BEC000844F750000000600C70ADE00F107B200CB
:10BED000F50FB20008003200E1CF4200020032004C
:10BEE0000170A00024000500810F700001003200E5
:10BEF0000408050044000500810F700002003A00AC
:10BF0000140005008502E9000000400081C04800DF
:10BF1000FCFF3B000170A000240005000080FA0037
:10BF2000000006000000FA0014002000C4FF070013
:10BF30000080FA00000006000000FA00020007007E
:10BF40000461040000000000889FBE008A9FBE00BC
:10BF50008C1F780059000700600033006450E10036
:10BF60004F0032006420E1005200320003826C0076
:10BF700007003B000905D0000306D000820F5400E3
:10BF80000C065D00020039000200320089017800D1
:10BF9000030678008582550004003D000003FD0083
:10BFA0008103FD008502EA008B854200840F720048
:10BFB00002003B0060001000E08018006011B80033
:10BFC0000005EB007A28E1000A003900060078003D
:10BFD000C75DDD00F707B200878075002D003700D0
:10BFE000828171000A017800610560008180D100C2
:10BFF0000080D3008502E900F9FF3B000604400001
:10C000008784480002003B0060041400E0841C00A8
:10C010000988A300070032008A81710082817100C3
:10C02000610164008904D1000884D3008B05E80015
:10C03000170037000978A30013003A000B00E00056
:10C04000130034008B05E9000804440089844C0087
:10C050000A4474000978A3000D003A000B00E000C8
:10C06000070034008B05E9000804440089844C0073
:10C0700001003A000B0020000978A300F7FF32000E
:10C080000001EB0002003700828171000A01780094
:10C09000220007000CF0A70001F0A00018003700F4
:10C0A0006420E10002003A00838F6C001800330026
:10C0B0000801BE000200BE00110037000004BE00EF
:10C0C0003C0007000003BE000405BE000200BE00E5
:10C0D00038000700844F7500000006000200BE0013
:10C0E0006450E100050036006420E10002003600E3
:10C0F0000968A30001003A000800BE000160A0002A
:10C100004F0678004F05BE004F04BE000000060039
:10C11000F0FF2F00F1FF2700F9FF3700810020001A
:10C12000618055000B003D000B00200061FE2F00D8
:10C130000100E1001D003400828171006101640092
:10C140008904D1000884D3000000E800FAFF3A0017
:10C1500071002000610064000300700002006000B4
:10C160000900320061044400E0844C000988A50005
:10C17000050032008B05E8006808E10002003A0083
:10C180008904D1000884D300F20F20000258E10096
:10C1900005003D00C75DDD00F907B200898075002C
:10C1A00008007800000006000BF827008B007800DC
:10C1B00000000500C70ADE00F107B200F50FB2006B
:10C1C00008003200E1CF4200020032000170A000FE
:10C1D00024000500810F70000100320004080500F2
:10C1E00044000500810F700002003A0014000500B1
:10C1F0008502E9000000400081C04800FCFF3B00D0
:10C200000170A000240005000080FA000000060074
:10C210000000FA00020007003A620400000000007B
:10C22000889FBE008A9FBE008C1F78003E000700DA
:10C230004500330003866C006450E1002E0032009C
:10C240006420E100330032006150E1002F00320031
:10C250006120E1003100320085855500EB07B00018
:10C2600009002000080420000500370008044400ED
:10C2700089844C000A0031000603430087834B0089
:10C280000001530081815B00F8FF33000203BE0010
:10C290000800A0000804440089844C00F6FF39001F
:10C2A000C639DD0083017300010032001300200055
:10C2B0008904D1000884D3000998A3000500320046
:10C2C0000800A7000300A0008904D1000884D3005F
:10C2D0008B05E8008904D1000884D3000001EB003D
:10C2E0000281D2002800070001F0A1000CF0A70095
:10C2F00001F0A0001D0037006420E1001F003200A3
:10C300000801BE000200BE00F7FF37006120E10017
:10C310001A0032006000B800F3FF37000000200070
:10C3200001F82700F0FF37000004BE003C000700C2
:10C330000003BE000405BE000200BE003800070076
:10C34000844F7500000006000200BE006450E1004A
:10C35000050036006420E100020036000968A300F1
:10C3600001003A000800BE000160A0004F067800FE
:10C370004F05BE004F04BE0000000600F0FF2F0076
:10C38000F1FF2700F9FF3700810020006180550090
:10C390000B003D000B00200061FE2F000100E100BA
:10C3A0001D00340082817100610164008904D100A4
:10C3B0000884D3000000E800FAFF3A007100200072
:10C3C0006100640003007000020060000900320098
:10C3D00061044400E0844C000988A5000500320097
:10C3E0008B05E8006808E10002003A008904D100EA
:10C3F0000884D300F20F20000258E10005003D0040
:10C40000C75DDD00F907B20089807500080078007B
:10C41000000006000BF827008B00780000000500E4
:10C42000C70ADE00F107B200F50FB20008003200C3
:10C43000E1CF4200020032000170A000240005009C
:10C44000810F70000100320004080500440005005F
:10C45000810F700002003A00140005008502E90017
:10C460000000400081C04800FCFF3B000170A000BC
:10C47000240005000080FA00000006000000FA0019
:10C48000020AB800800278000200B8008100420071
:10C49000032AB800810042000080FA000000060074
:10C4A0000F802000E0BF2000000188004440A80069
:10C4B00000002000A001880080ED2000C15B2F005B
:10C4C000C3000900315878009000FA00600047006E
:10C4D00041552F000E000900315878006F004700C9
:10C4E00031562F002C00090031587800C00320007D
:10C4F0000000470001592F0018000900315878004A
:10C500005005200000004700915A2F000300090049
:10C51000315878009005200000004700D15A2F00C4
:10C520000500090031587800F005200000004700A0
:10C53000315B2F000700090031587800000020000F
:10C5400040379800000020007037980000772000E6
:10C55000400E880000002000C0168800E4FF2F0075
:10C56000A02D200010086200E0E02000801F78006D
:10C5700010002000801F780032FD07004F00B1003E
:10C5800014002000A02D200010087200002C2100B3
:10C5900001002000801F7800811F7800B4D00700C0
:10C5A0004F00B10004402000C0202000100872009D
:10C5B00000102E0001002000801F7800811F7800ED
:10C5C00044D107004F00B100040028006021200082
:10C5D0001008720040F92000C062880060EA200064
:10C5E000CF80DE00B0688800C168880060EA200063
:10C5F0000100200090688800A168880060EA20009F
:10C6000001002000306888004168880060EA20004E
:10C610000100200070688800816888000000200008
:10C62000100E8800701A2600200E88008000280056
:10C63000000E880060EA2000D00E8800D00E800036
:10C64000C00E8800C00E8000B00E880000002000E0
:10C6500010688800000020000068880000002000AA
:10C660002068880075D107008BD1070000002000EA
:10C67000CF80DE001069880021698800003A8000C0
:10C68000700060004402DE000400E00032003A0066
:10C690000000200001002000806F8800916F88005A
:10C6A0000000200001002000406F8800516F8800CA
:10C6B0000000200001002000606F8800716F88007A
:10C6C000000020002070880000002000107088000A
:10C6D0000000200000708800000020000100200001
:10C6E000F072880001738800000020000100200023
:10C6F000D0728800E1728800000020000100200054
:10C70000B0728800C1728800000020000100200083
:10C7100090728800A172880000002000CF80DE00A7
:10C7200080698800916988000000200030708800CE
:10C73000A0C52F00F10720002087980031879800BE
:10C7400000002000CF80DE004087980051879800CD
:10C75000000020006037980000002000F070880082
:10C7600000002000E0708800000020003071880088
:10C77000000020000071880000002000CF80DE0053
:10C780000081EB00BCFC0700C0718800D1718800FB
:10C7900000002000CF80DE00F07388000174880064
:10C7A0000000200001002000D0738800E1738800A1
:10C7B0000000200001002000B0738800C1738800D1
:10C7C000000020000100200090738800A173880001
:10C7D0000000200001002000707288008172880033
:10C7E0000000200001002000506B8800616B880071
:10C7F00000002000010020001071880021718800D5
:10C800000000200001002000407188005171880064
:10C810000000200001002000706B8800816B880000
:10C8200000002000010020008070880091708800C6
:10C830000000200001002000006B8800116B8800C0
:10C840000000200001002000E06A8800F16A8800F2
:10C850000000200001002000906A8800A16A880082
:10C860000000200001002000C06A8800D16A880012
:10C870000000200001002000603F9800713F9800F8
:10C880000000200001002000403F9800513F980028
:10C890000000200001002000607088007170880096
:10C8A0000000200001002000A0708800B170880006
:10C8B00000002000010020004070880051708800B6
:10C8C00000002000706A880000002000806A880054
:10C8D0000000200001002000203F9800313F980018
:10C8E0000000200001002000506A8800616A880072
:10C8F000000020000069880000002000F068880027
:10C9000000002000E068880000002000D068880057
:10C9100064D5200000022000004A780074D5200071
:10C9200000022000004A780054D3200000022000BA
:10C93000004A7800000020004073880000002000BA
:10C94000103F980000002000003F980000002000E9
:10C95000D070880000002000406B8800000020009C
:10C96000906B8800000020002073880000002000E9
:10C970000072880000002000107388000000200072
:10C9800050698800000020003073880000002000FB
:10C990005068880000002000403798008006200082
:10C9A00000004700100278006C00520016003D00A5
:10C9B0008606200006034700160078004202DD00CC
:10C9C00040D720000402400000002000000A780048
:10C9D00006007800100078004202DD0040D72000F9
:10C9E000040040006202400000002000000A7800BD
:10C9F00014002000800620000000470010084200BC
:10CA0000CE64040000000000000020007071880067
:10CA1000000020006071880000002000B0718800D4
:10CA2000000020009071880000002000A0718800A4
:10CA3000000020008071880000002000E062880073
:10CA400000002000F062880010002000006F8800C5
:10CA5000100020006068880044D3200040002000BF
:10CA6000004A780000102000801F7800000020009D
:10CA7000801F780000002000801F78000000200048
:10CA8000801F780000002000801F78002000200018
:10CA9000801F780000002000801F78000002200026
:10CAA000801F780025D107000F01B10000C02F00C2
:10CAB000F1072000008798001187980000002000EF
:10CAC00040379800800620000000470010027800E0
:10CAD0007B00520014003D0080062000000047004B
:10CAE000100078004202DD0080F2200004024000C5
:10CAF00062004200901F7800941F78000008200018
:10CB000000004700801F780057D307006F00B10076
:10CB1000140020008006200000004700100842009A
:10CB2000626504000000000090628000C070880010
:10CB3000646080006000520008003500A6D7200025
:10CB4000CFB3DE00E4D020003400130024801B00AB
:10CB500002003500626604000000000000002000B2
:10CB60000124240030618800416188000000200019
:10CB700001222400D0608800E160880000002000CD
:10CB800001172400F0608800016188000000200087
:10CB90000112240090608800A1608800000020003D
:10CBA000011024001061880021618800000020002D
:10CBB00001002000B0608800C160880000002000F3
:10CBC000010A240050618800616188000000200093
:10CBD0004123240090618800A161880000002000AA
:10CBE00001122400B0618800C1618800B0042000F7
:10CBF0006060880000002400C15924007060880033
:10CC0000816088006066260061FA23004060880029
:10CC10005160880010002000F061880010002000A2
:10CC20000062880000002000812C240070618800D0
:10CC30008161880000002800414D2400D0618800F7
:10CC4000E161880090C22500F1D8230020608800AF
:10CC500031608800000020006149240000608800E5
:10CC600011608800100020001062880080072000FA
:10CC700020628800100020003062880050002000F0
:10CC800040628800D0192E00C1BB2300506288008A
:10CC900061628800207C210061DA230070628800D4
:10CCA0008162880000002000C07088000000200021
:10CCB0009062880000002000A06288000000200030
:10CCC000B062880000002000010E2400E07188009E
:10CCD000F171880000002000010E240030728800ED
:10CCE00041728800D0688000CF80DE000081EB00B8
:10CCF00061FB0700B2FA2C0053CD2300B9FB0700FB
:10CD00006087980071879800C0718800D171880091
:10CD1000E0688000CF80DE000081EB0056FB07005A
:10CD200012362C0033CD2300AEFB070010728800B2
:10CD3000217288006E809000FE80900000027800D2
:10CD40008102780000002000811024000401780096
:10CD50008501780030FC07000000E00002003C0084
:10CD60000000200001003700100020000000E0005B
:10CD70000600320000002000010E2400E07188004F
:10CD8000F1718800CE660400000000000000200061
:10CD900001122400E0718800F17188001472800093
:10CDA000257280000000200081102400040178001A
:10CDB0008501780018FC07000000E00002003C003C
:10CDC0000000200001003700100020000000E000FB
:10CDD0000600320000002000010E2400307288009E
:10CDE0004172880026670400000000001472800071
:10CDF00025728000D0CC2C00C114240004017800DE
:10CE00008501780004FC07000000E00002003C00FF
:10CE10000000200001003700100020000000E000AA
:10CE20000600320000002000011224003072880049
:10CE30004172880026670400000000000000200006
:10CE40000115240030728800417288004060800023
:10CE500051608000106F8800216F88006060800042
:10CE6000306F88006460800060DE2000610842004E
:10CE7000E06A2000801F7800700B2000801F78007F
:10CE8000F0FA07004F00B10030E80700460CF80048
:10CE900080532F00801F780089F507004F00B100F4
:10CEA00060004700801F78006AF507002F00B1007E
:10CEB000E0462000801F7800A0072000801F780037
:10CEC000E0FA07004F00B10096F507006F00470039
:10CED000801F78005FF507002F00B100E01E2100E1
:10CEE000801F7800801E2000801F7800D5FA070080
:10CEF0004F00B1002000200040379800800620003D
:10CF00000000470010027800600052001800340052
:10CF100080062000000047001000780061005000EB
:10CF200040379800801F780010542F00801F780031
:10CF300040DA2000801F780090EA07006F00B100FF
:10CF400040DA2000801F78007BD507002F00B10059
:10CF5000E0CE2200801F7800404C2000801F780027
:10CF6000B8FA07004F00B1007E670400000000001F
:10CF7000F6E7070004402000E020200010087200BF
:10CF800004002800C02020001008720010082000B3
:10CF9000801F780009D007002F00B1005001200049
:10CFA000801F780005D007002F00B100000220008C
:10CFB000801F780001D007002F00B100F4DF2F00A0
:10CFC0004008200010086200D4FF2F00E02020005D
:10CFD00010086200C003200000004700801F780096
:10CFE00055D507002F00B1000ED007006002500099
:10CFF00002003500F46704000000000021D00700A3
:10D000000004E00003003A000060FE00FE67040038
:10D0100000000000E08E2000801F7800400F2000FC
:10D02000801F780087FA07004F00B100C7E70700AC
:10D030003CF507005005200000004700801F7800E5
:10D0400088EA07002F00B100E0462000801F78002A
:10D05000A0072000801F78007AFA07004F00B10077
:10D06000003A8000700060004402DE000400E0002E
:10D070000600320000002000801F7800C2EA07008E
:10D080002F00B1004E6804000000000010002000D6
:10D09000801F7800BCEA07002F00B10000002000CC
:10D0A000003A8800E0462000801F7800A00720009A
:10D0B000801F780063FA07004F00B1009005200040
:10D0C00000004700801F780066EA07002F00B100CB
:10D0D000F005200000004700801F780061EA07008B
:10D0E0002F00B10000002000403798000000200011
:10D0F00070379800540CF800CBEA07002F00B100FD
:10D10000E0CF07000004E000C50132000060FE002F
:10D11000C4CF07005037980060025000BE013500B0
:10D120004605200084062000040247001400130076
:10D130000600340000002000403798000000200066
:10D14000703798000C6C040000000000EA6B0400CB
:10D150000000000000002000403798001000200070
:10D16000703798000C6C04000000000020E82000DC
:10D17000860620000603470016024000000020003B
:10D18000004A780010002000160B40000C6C0400D0
:10D190000000000024E82000800620000000470076
:10D1A0001002420000002000004A7800E006200043
:10D1B0000000470010027800600052007201320047
:10D1C000000020007037980020E82000801F7800C1
:10D1D000D3D107002F00B100600250006A01340073
:10D1E000746B8000856B8000826F8000936F80007D
:10D1F00004007800850078000CFB07008070880030
:10D20000917088004007200000004700300278003D
:10D21000A0027800506A8000616A800004017800F2
:10D22000850178003FFB07000000E00002003A00A3
:10D230000000200001003700100020000000E00086
:10D240008E003200400720000000470030027800C6
:10D25000A0027800506A8000616A800004017800B2
:10D26000850178002FFB07000000E0000200350078
:10D270000000200001003700100020000000E00046
:10D280000B00320040072000000047003002780009
:10D29000A002780002002000032724000400780088
:10D2A00085007800E1FA0700203F9800313F9800A0
:10D2B0001400200000072000000047001008420072
:10D2C0001400200020072000000047001008420042
:10D2D0008670800097708000840720000402470059
:10D2E00034017800A40178000600780087007800F7
:10D2F000CEFA07001071880021718800066B80004B
:10D30000176B8000C4072000040247003401780036
:10D31000A40178000600780087007800C3FA0700AF
:10D320004071880051718800000278008102780005
:10D3300000002000413324000401780085017800BA
:10D34000F8FA07000000E0000200350000002000AD
:10D3500001003700100020000000E0000B00320048
:10D36000447180005571800002002000433B24007E
:10D370000400780085007800ACFA0700407188004E
:10D3800051718800F46904000000000044718000BD
:10D39000557180000000200041332C00040178000A
:10D3A000850178009CFA07000000E00002003C00C4
:10D3B0000000200001003700100020000000E00005
:10D3C0000900320044718000557180000000200087
:10D3D000413B24000401780085017800D6FA07005B
:10D3E0004071880051718800566A8000676A800029
:10D3F000440720000402470034017800A4017800AB
:10D40000060078008700780088FA07006087980097
:10D4100071879800000178008101780040718000D8
:10D42000517180007AFB07004071880051718800BB
:10D430006E819000FE81900010718000217180004B
:10D4400073FB07001071880021718800506A80000A
:10D45000616A8000203F9800313F98008070800012
:10D4600091708000403F9800513F9800006B800011
:10D47000116B8000603F9800713F9800347080000D
:10D480006000520003003A0042D40700C46B04005D
:10D490000000000000002000801F7800CCD80700AA
:10D4A0002F00B100446B800063005200360034004E
:10D4B000E46A8000F56A800090728000A1728000AA
:10D4C000040178008501780096FA07000000E0006A
:10D4D000020035000000200001003700100020008D
:10D4E0000000E00004003200E06A8000F16A800081
:10D4F00090728800A172880064708000757080004E
:10D50000D0728000E172800004017800850178000B
:10D5100084FA07000000E00002003500000020004F
:10D5200001003700100020000000E000040032007D
:10D530006070800071708000D0728800E172880095
:10D540008470800095708000B0728000C17280008D
:10D55000040178008501780072FA07000000E000FD
:10D5600002003500000020000100370010002000FC
:10D570000000E000040032008070800091708000A4
:10D58000B0728800C1728800646880006000520038
:10D590000C003A00546880006000520009003A0014
:10D5A0000007200000004700901F780010002000B6
:10D5B000801F7800CBD907004F00B100F06A04004B
:10D5C000000000000007200000004700901F7800C6
:10D5D00000002000801F7800C2D907004F00B10072
:10D5E00000002000003F980044628000600052006C
:10D5F0006500340020072000000047001003780079
:10D6000084C42000140053005F0035000000200097
:10D61000103F9800E46A8000F56A80000000200056
:10D6200001F0230004017800850178003DFA07002D
:10D630000000E0000200340000002000010037007C
:10D64000100020000000E00007003A00C0062000A3
:10D650000000470010027800600052000200320013
:10D66000C46B0400000000004008200000004700D8
:10D6700030037800A003780044FF2F00F507200056
:10D680000400530005805B003F003E00002424009E
:10D69000F1002000726A8000CF91DE0077FB070066
:10D6A00046D6200036024000A682480064879800D3
:10D6B0007587980000102E00515F2000826A80005C
:10D6C000CF91DE006DFB07006E829000FE8290001D
:10D6D0000002420081824A008008200000004700CA
:10D6E0001018420010904A00C006200000004700B9
:10D6F000100278006000520018003A00200020005C
:10D70000CF80DE004408200004024700141A1000F5
:10D710001492180010002000801F7800C00620001E
:10D7200000004700801F7800841F780096E90700FA
:10D730006F00B10020002000801F780080082000CA
:10D7400000004700801F78004008200000004700CC
:10D75000801F78008CE907006F00B100C006200030
:10D76000000047001000780061004000603798001A
:10D77000801F78004008200000004700801F7800CC
:10D7800010DB07004F00B1000C6C0400000000002B
:10D79000E006200000004700100278006000520000
:10D7A0000A00320020E82000860620000603470019
:10D7B00016024000A006200000004700104078003C
:10D7C000004A780010002000160B40000C6C04008A
:10D7D0000000000046022000A406200004024700CA
:10D7E000140013005BFE3200A0062000000047007A
:10D7F000100278006D0052005CFE3200A00620008E
:10D8000000004700100278006A00520061FE3200FA
:10D81000C86B0400000000008068040000000000E5
:10D8200040D320001042780061405200B50039001A
:10D83000EBF207000608200006025000B100390094
:10D8400044D3200000002000004A7800D068800007
:10D85000CF80DE000081EB0087F80700B2FA2C00D1
:10D8600053CD2300DFF80700C4718000D57180001C
:10D870000401780085017800AFF90700020020005C
:10D880000300240062FA0700C0718800D17188008B
:10D89000E0688000CF80DE000081EB0076F80700B2
:10D8A00012362C0033CD2300CEF80700147280000E
:10D8B0002572800004017800850178009EF9070038
:10D8C000020020000300240051FA070010728800B3
:10D8D0002172880060698000CF80DE000081EB004B
:10D8E00065F807007262800083628000BDF807005F
:10D8F000507288006172880000027800810278000E
:10D90000F0728000017380000401780085017800C6
:10D9100084F907000000E00002003500000020004C
:10D9200001003700100020000000E0000400320079
:10D930005072800061728000F0728800017388006C
:10D9400080698000916980000001EB004AF80700BF
:10D950005262800063628000A2F807007072880043
:10D960008172880006AF2000CFB3DE0024D12000F2
:10D970003400130024801B0014003D003070800030
:10D980000000E00011003200546880006100520085
:10D9900007003A00000020005068880010002000B6
:10D9A000906B880069E50700E26C0400000000004D
:10D9B000000020006068880010002000006F8800D0
:10D9C00054DD0700806D04000000000010002000FE
:10D9D00060688800C63E2100CFB3DE0024D120005D
:10D9E0003400130024801B000400340060EA20008F
:10D9F000CF80DE0090688800A1688800C6252100DD
:10DA0000CFB3DE0024D120003400130024801B009B
:10DA100008003400046F80006100520003003A00E7
:10DA20004AE5070000002000006F8800806D0400B8
:10DA30000000000046192100CFB3DE0024D12000F1
:10DA40003400130024801B0017003400046F800092
:10DA50006100520003003A003CE50700000020008E
:10DA6000006F880054688000600052000B003A008C
:10DA70001000200050688800706880008168800075
:10DA800050738800617388003068800041688000AE
:10DA90007073880081738800A6E70700A6F207006C
:10DAA000806D040000000000546880006100520096
:10DAB00005003A00000020005068880023E50700B8
:10DAC000806D04000000000010002000006F88003E
:10DAD000A06280000000E00008003200C410800056
:10DAE00000202000000062004902DE000400E00087
:10DAF00002003A0010062000D010880005DD070063
:10DB000037F2070080680400000000000080FA007F
:10DB1000FFFF37003235FF00312CFF003338FF00A4
:10DB20003430FF003000FF000000FF000000FF0065
:10DB30000000FF000000FF000000FF000000FF00E9
:10DB40000000FF000000FF000000FF000000FF00D9
:10DB50003C0AFF002530FF003130FF006C75FF00EC
:10DB60000A00FF002538FF002E36FF00662CFF005C
:10DB70002538FF002E36FF00662CFF002564FF00CD
:10DB80000A00FF004750FF00524DFF004300FF0016
:10DB90004750FF004747FF004100FF004750FF008C
:10DBA0004753FF005600FF005049FF004E47FF005B
:10DBB0000050FF004F4EFF00470AFF000047FF00E4
:10DBC0004554FF004C4FFF004700FF003E0AFF0096
:10DBD0000053FF006574FF007469FF006E67FF006B
:10DBE0002048FF004F4DFF004520FF00252DFF007E
:10DBF0003364FF000048FF004F4DFF004520FF0049
:10DC00006E6FFF007420FF007365FF007400FF005B
:10DC10000000FF000000FF00C4FFFF007F3FFF0087
:10DC200080EFFF00FFBEFF0090E1FF00A93EFF0074
:10DC3000EC82FF0076BEFF0082ADFF002B3EFF00AE
:10DC40000E3CFF00C3BDFF0087D1FF00133DFF0066
:10DC50004178FF00D3BBFF000000FF00803FFF00C2
:10DC60001872FF00313FFF00F0FDFF00753EFF001E
:10DC70004758FF00633DFF005895FF001D3CFF0023
:10DC800082C4FF00AE3AFF00A878FF002139FF00F0
:10DC9000EF93FF008037FF00A092FF00A735FF0041
:10DCA0004656FF001534FF00063CFF000442FF000B
:10DCB0007D9FFF006A42FF005C90FF000142FF0071
:10DCC000604DFF00BB40FF0051ECFF00473EFF00EE
:10DCD000DE8DFF001FBBFF00063CFF000442FF007B
:10DCE000C059FF008B42FF007404FF004442FF0054
:10DCF000F99BFF004F41FF000000FF00803FFF0045
:10DD00001B5BFF003958FF00001BFF005B37FF0063
:10DD1000396DFF004155FF00544FFF005049FF008F
:10DD20004C4FFF005400FF001B5BFF00307AFF00E8
:10DD30001B5BFF002564FF003B25FF006478FF00AC
:10DD4000001BFF005B34FF007A1BFF005B25FF0018
:10DD5000643BFF002564FF007800FF00ECF3FF0048
:10DD60004A48FF003595FF0095C7FF0017C1FF0027
:10DD7000DC45FF00FDDBFF006DC3FF0072B3FF0059
:10DD80003340FF002B34FF000148FF007F9DFF0060
:10DD9000B045FF00E7FFFF00D942FF000000FF0091
:10DDA000803FFF001B5BFF00302FFF007200FF0071
:10DDB0001B5BFF002564FF003B25FF00642EFF0076
:10DDC0007200FF001B5BFF002564FF003B25FF0086
:10DDD000642DFF007200FF001B5BFF002F72FF002D
:10DDE000001BFF005B30FF007A1BFF005B25FF007C
:10DDF000643BFF002564FF004800FF002530FF0062
:10DE00003264FF003A25FF003032FF00641BFF0040
:10DE10005B34FF007A25FF003032FF006420FF00F2
:10DE20005554FF004300FF002530FF003264FF001F
:10DE30003A25FF003032FF00641BFF005B34FF0017
:10DE40007A25FF003032FF006400FF002523FF0029
:10DE5000362EFF003166FF001B5BFF00317AFF00AA
:10DE60006B70FF006800FF002523FF00362EFF00C7
:10DE70003166FF001B5BFF00317AFF006D70FF0011
:10DE80006800FF002523FF00362EFF003166FF00EB
:10DE90001B5BFF00317AFF006D00FF002523FF00B0
:10DEA000362EFF003166FF001B5BFF00317AFF005A
:10DEB0006674FF00001BFF005B30FF007A25FF0047
:10DEC0006325FF006300FF002523FF00352EFF00C0
:10DED0003266FF001B5BFF00317AFF005600FF0037
:10DEE0001B5BFF00307AFF002535FF002E30FF005E
:10DEF000661BFF005B31FF007A43FF00001BFF0041
:10DF00005B30FF007A25FF00352EFF003066FF00F2
:10DF10001B5BFF00317AFF004600FF001B5BFF0028
:10DF2000307AFF001B5BFF003758FF000025FF0021
:10DF30002335FF002E32FF00661BFF005B31FF0020
:10DF40007A56FF001B5BFF003639FF006D1BFF0098
:10DF50005B34FF007A20FF004558FF005400FF00AB
:10DF60002523FF00352EFF003166FF001B5BFF00FD
:10DF7000317AFF004100FF002535FF002E30FF0001
:10DF8000661BFF005B31FF007A6DFF004168FF00F8
:10DF90000025FF00352EFF003066FF001B5BFF00F1
:10DFA000317AFF006D00FF002523FF00352EFF00B2
:10DFB0003266FF001B5BFF00317AFF006D6CFF00D3
:10DFC0000025FF00352EFF003066FF001B5BFF00C1
:10DFD000317AFF006674FF000025FF00352EFF0038
:10DFE0003066FF001B5BFF00317AFF006D00FF0011
:10DFF0002523FF00352EFF003266FF001B5BFF006C
:10E00000317AFF006D6CFF000025FF00352EFF0008
:10E010003066FF001B5BFF00317AFF006674FF0073
:10E02000001BFF005B34FF007A53FF005045FF00E8
:10E030004544FF00201BFF005B30FF007A25FF00F6
:10E040002336FF002E31FF00661BFF005B31FF000F
:10E050007A6BFF007068FF00001BFF005B34FF005D
:10E060007A20FF002041FF004C54FF00201BFF00DE
:10E070005B30FF007A25FF002336FF002E31FF00C2
:10E08000661BFF005B31FF007A6DFF00001BFF0085
:10E090005B34FF007A52FF00414EFF004745FF000E
:10E0A000201BFF005B30FF007A25FF00362EFF00AB
:10E0B0003066FF001B5BFF00317AFF006D00FF0040
:10E0C0001B5BFF00347AFF005350FF004545FF0003
:10E0D0004420FF001B5BFF00307AFF002523FF0078
:10E0E000362EFF003166FF001B5BFF00317AFF0018
:10E0F0006D70FF006800FF001B5BFF00347AFF00BB
:10E100002020FF00414CFF005420FF001B5BFF005C
:10E11000307AFF002523FF00362EFF003166FF0016
:10E120001B5BFF00317AFF006674FF00001BFF00DD
:10E130005B34FF007A52FF00414EFF004745FF006D
:10E14000201BFF005B30FF007A25FF002336FF0015
:10E150002E32FF00661BFF005B31FF007A6DFF006F
:10E160006C00FF001B5BFF00347AFF002043FF00C0
:10E170005552FF005220FF001B5BFF00307AFF006A
:10E180002523FF00362EFF003166FF001B5BFF00DA
:10E19000317AFF004100FF001B5BFF003635FF00B6
:10E1A0006D25FF003264FF001B5BFF003639FF0066
:10E1B0006D1BFF005B34FF007A20FF005341FF001E
:10E1C0005453FF000025FF003264FF001B5BFF007B
:10E1D000347AFF002053FF004154FF005300FF003A
:10E1E0002523FF003130FF002E36FF00661BFF00A5
:10E1F0005B34FF007A25FF006300FF002523FF004A
:10E200003130FF002E36FF00661BFF005B34FF003D
:10E210007A25FF006300FF001B5BFF00347AFF00DC
:10E220004844FF004F50FF00201BFF005B30FF0001
:10E230007A25FF00232DFF00362EFF003166FF00F8
:10E240000025FF003033FF006400FF002025FF00A1
:10E250007320FF00001BFF005B37FF00346DFF00E1
:10E260002530FF00332EFF003066FF000025FF0041
:10E270003033FF002E30FF006600FF00201BFF0040
:10E280005B37FF00316DFF002573FF001B5BFF0054
:10E290003639FF006D20FF000020FF002573FF00CE
:10E2A0002000FF002025FF007320FF0000C4FF00B6
:10E2B0002563FF001B5BFF00347AFF00201BFF007B
:10E2C0005B30FF007A00FF00C425FF00631BFF00E6
:10E2D0005B34FF007A20FF001B5BFF00307AFF00F9
:10E2E0000025FF003032FF006420FF00001BFF000C
:10E2F0005B38FF005800FF001B5BFF003658FF0033
:10E30000001BFF005B37FF005800FF001B5BFF0096
:10E310003758FF00001BFF005B34FF007A4CFF0002
:10E320004F53FF00201BFF005B30FF007A00FF000F
:10E330005045FF00414BFF002056FF00414CFF00BD
:10E340005545FF005300FF001B5BFF003131FF000C
:10E350005800FF001B5BFF003132FF005800FF0038
:10E360001B5BFF003132FF005800FF001B5BFF000A
:10E370003132FF005800FF001B5BFF003132FF000D
:10E380005800FF001B5BFF003958FF00001BFF0017
:10E390005B35FF005800FF001B5BFF003131FF00C1
:10E3A0005800FF001B5BFF003131FF005800FF00E9
:10E3B0001B5BFF003958FF0000C0FF00A000FF00FA
:10E3C000C0A0FF0000C3FF00BF00FF00C480FF002B
:10E3D00000C0FF00A000FF00C480FF0000C3FF00DA
:10E3E000BF00FF00C0A0FF00001BFF005B34FF0068
:10E3F0007A00FF002D2DFF002000FF001B5BFF00B7
:10E40000324AFF00001BFF005B31FF007A1BFF0058
:10E410005B25FF00643BFF002564FF007800FF00E0
:10E42000204DFF004158FF005241FF004E47FF00C2
:10E430004520FF002020FF00201BFF005B30FF0075
:10E440007A25FF00362EFF003066FF002000FF0017
:10E45000204CFF004F57FF00414CFF005452FF007B
:10E460004154FF00494FFF00201BFF005B30FF00BD
:10E470007A25FF00362EFF003266FF002000FF00E5
:10E480002056FF00414CFF004944FF004844FF0074
:10E490004F50FF002020FF00201BFF005B30FF00DB
:10E4A0007A25FF00362EFF003166FF002000FF00B6
:10E4B000204DFF00494EFF005641FF004C49FF0030
:10E4C0004420FF002020FF00201BFF005B30FF00E6
:10E4D0007A25FF003664FF002000FF002053FF0074
:10E4E000484FFF005748FF004F4DFF00454CFF00CD
:10E4F000494DFF00201BFF005B30FF007A25FF0025
:10E50000362EFF003066FF002000FF002052FF0083
:10E510004F43FF004C49FF004D49FF005420FF00CE
:10E520002020FF00201BFF005B30FF007A25FF004A
:10E53000362EFF003166FF002000FF002052FF0052
:10E540004F43FF005354FF004550FF004741FF0079
:10E55000494EFF00201BFF005B30FF007A25FF00C3
:10E56000362EFF003066FF002000FF002041FF0034
:10E570005052FF004F43FF004741FF00494EFF004C
:10E580002020FF00201BFF005B30FF007A25FF00EA
:10E59000362EFF003166FF002000FF002052FF00F2
:10E5A0004F54FF004C49FF004D49FF005420FF002D
:10E5B0002020FF00201BFF005B30FF007A25FF00BA
:10E5C000362EFF003166FF002000FF002052FF00C2
:10E5D0004F54FF005354FF004550FF004741FF00D8
:10E5E000494EFF00201BFF005B30FF007A25FF0033
:10E5F000362EFF003066FF002000FF002041FF00A4
:10E600005052FF004F54FF004741FF00494EFF00AA
:10E610002020FF00201BFF005B30FF007A25FF0059
:10E62000362EFF003166FF002000FF002053FF0060
:10E630005045FF004544FF004C4FFF00574CFF0082
:10E64000494DFF00201BFF005B30FF007A25FF00D3
:10E65000362EFF003166FF002000FF002043FF0040
:10E660005255FF004953FF004541FF004C54FF0045
:10E670002020FF00201BFF005B30FF007A25FF00F9
:10E68000362EFF003066FF002000FF00204DFF0007
:10E690004158FF00414CFF005443FF004847FF0032
:10E6A0002020FF00201BFF005B30FF007A25FF00C9
:10E6B000362EFF003066FF002000FF00204DFF00D7
:10E6C0004158FF004844FF004743FF004847FF0010
:10E6D0002020FF00201BFF005B30FF007A25FF0099
:10E6E000362EFF003066FF002000FF00204DFF00A7
:10E6F0004148FF005741FF00524EFF00494EFF00C6
:10E700004720FF00201BFF005B30FF007A25FF0041
:10E71000362EFF003066FF002000FF002045FF007E
:10E720004C45FF005345FF005256FF004F44FF0089
:10E730004952FF00201BFF005B30FF007A25FF00DD
:10E740003673FF002000FF002052FF004452FF00FC
:10E750005345FF005256FF004F44FF004952FF004F
:10E76000201BFF005B30FF007A25FF003673FF009F
:10E770002000FF002055FF004E49FF005453FF00CA
:10E780002020FF002020FF002020FF002020FF008D
:10E790002538FF007320FF000020FF00414DFF00DF
:10E7A0005053FF005A45FF00524FFF002020FF004A
:10E7B0002020FF001B5BFF00307AFF002536FF00A2
:10E7C0006420FF000020FF005649FF004445FF0081
:10E7D0004F4DFF004F44FF004520FF002020FF0069
:10E7E0002025FF003873FF002000FF00204CFF00B1
:10E7F0004F47FF005045FF005249FF004F44FF00C4
:10E800002020FF00201BFF005B30FF007A25FF0067
:10E810003664FF002000FF002048FF004F4DFF003E
:10E82000454CFF004F43FF002020FF002020FF0049
:10E830002020FF002538FF007320FF000020FF008C
:10E840004D41FF00484DFF00554CFF005420FF0094
:10E85000201BFF005B30FF007A20FF002537FF0000
:10E860002E35FF006620FF000020FF00414DFF0015
:10E87000504DFF00554CFF005420FF002020FF00AA
:10E880002020FF001B5BFF00307AFF002536FF00D1
:10E890002E33FF006620FF000020FF005341FF00E1
:10E8A0004645FF005A4FFF004E45FF002020FF0065
:10E8B0002020FF001B5BFF00307AFF002536FF00A1
:10E8C0006420FF000020FF00564FFF004C54FF0063
:10E8D000314CFF004F57FF004152FF004E20FF0018
:10E8E0001B5BFF00307AFF002536FF007320FF001E
:10E8F0000020FF004452FF004157FF00484FFF0037
:10E900005249FF005A4FFF004E20FF001B5BFF00E3
:10E91000307AFF002536FF007320FF000020FF0043
:10E920005341FF005645FF002043FF004F4EFF00BC
:10E930004649FF004720FF001B5BFF00307AFF00C5
:10E940002536FF007320FF00004EFF004F52FF00EE
:10E950000052FF004556FF00004EFF004F52FF00DF
:10E960000052FF004556FF00004DFF004554FF00D8
:10E970005249FF004300FF00494DFF005045FF0092
:10E980005249FF00414CFF000050FF00414CFF0086
:10E99000004EFF005453FF004300FF005345FF00AB
:10E9A0005400FF00554EFF005345FF005400FF0088
:10E9B0004F46FF004600FF00204FFF004E00FF00C3
:10E9C0004F4EFF000020FF004F46FF004600FF00B3
:10E9D0002A00FF00444FFF004E45FF000025FF00C6
:10E9E0003032FF007800FF002450FF004D54FF003C
:10E9F0004B25FF00732AFF002573FF000D0AFF005F
:10EA00000033FF003134FF002C30FF002C31FF00B9
:10EA10002C30FF002C31FF002C30FF002C00FF00B9
:10EA20003100FF003000FF002C30FF002C30FF00D1
:10EA30002C30FF002C30FF002C30FF002C30FF006A
:10EA40002C30FF002C30FF002C30FF002C30FF005A
:10EA50002C30FF00003CFF004E55FF004C4CFF00E7
:10EA60003E00FF001B5BFF002564FF006D00FF0000
:10EA70001B5BFF003136FF003B25FF006476FF0083
:10EA80000047FF005053FF002F4FFF005344FF008B
:10EA90002053FF005441FF005254FF005550FF0027
:10EAA0002025FF006400FF001B5BFF003231FF00E8
:10EAB0003B30FF00761BFF005B33FF00323BFF0063
:10EAC0003176FF00001BFF005B31FF007A44FF003E
:10EAD0007261FF00676FFF006E4FFF005344FF003D
:10EAE0002056FF00342EFF00386BFF002032FF005D
:10EAF000322FFF00312FFF003230FF003039FF008E
:10EB00002028FF006329FF002044FF00616EFF0002
:10EB10006965FF006C20FF005765FF006500FF007E
:10EB20005761FF006974FF00696EFF006720FF00F6
:10EB3000666FFF007220FF004750FF005320FF0068
:10EB40006461FF007461FF00202EFF002E2EFF0085
:10EB50000030FF003030FF000033FF003031FF0095
:10EB60002C32FF000032FF003230FF002C32FF0059
:10EB70003030FF0000FFFF003031FF003233FF0074
:10EB80003435FF003637FF003839FF006162FF007F
:10EB90006364FF006566FF006768FF00696AFF0045
:10EBA0006B6CFF006D6EFF006F70FF007172FF00F5
:10EBB0007374FF007576FF007778FF00797AFF00A5
:10EBC00000FFFF00D80EFF003031FF003233FF009E
:10EBD0003435FF003637FF003839FF004142FF006F
:10EBE0004344FF004546FF004748FF00494AFF00F5
:10EBF0004B4CFF004D4EFF004F50FF005152FF00A5
:10EC00005354FF005556FF005758FF00595AFF0054
:10EC100000FFFF00000FFF00000CFF000200FF00DC
:10EC2000040CFF000200FF00080CFF000200FF00C0
:10EC30000C0CFF000100FF000E0CFF000200FF00A3
:10EC4000120CFF000200FF00160CFF000200FF0084
:10EC50001A0CFF000200FF001E0CFF000200FF0064
:10EC6000220CFF000200FF00260CFF000200FF0044
:10EC70002A0CFF000200FF002E0CFF000200FF0024
:10EC8000320CFF000200FF00360CFF000200FF0004
:10EC90003A0CFF000200FF003E0CFF000100FF00E5
:10ECA000400CFF000100FF00420CFF000100FF00CC
:10ECB000440CFF000100FF00460CFF000100FF00B4
:10ECC000480CFF000100FF004A0CFF000200FF009B
:10ECD0004E0CFF000200FF00520CFF000100FF007D
:10ECE000540CFF000100FF00560CFF000100FF0064
:10ECF0000000FF000000FF000000FF000000FF0018
:0200000401F009
:10000000F6FF0000F4FF00007F7A0000FFFFFF0012
:0C001000FFFFFF00FFFF0000FFFF0000EB
:00000001FF
